:020000040800f2
:200000000050002015020008590200085b0200085b0200085b0200085b020008000000005a
:020000040800f2
:20002000000000000000000000000000590200085902000800000000590200085902000834
:020000040800f2
:20004000590200085902000859020008590200085902000859020008590200085902000888
:020000040800f2
:20006000590200085902000859020008590200085902000859020008590200085902000868
:020000040800f2
:2000800059020008590200085902000859020008fd0800085902000859020008590200089e
:020000040800f2
:2000a000590200085902000859020008590200085902000859020008590200085902000828
:020000040800f2
:2000c000590200085902000859020008590200085902000859020008590200085902000808
:020000040800f2
:2000e0005902000859020008f5090008590200085902000859020008590200085902000845
:020000040800f2
:200100005902000859020008590200085902000859020008590200085902000859020008c7
:020000040800f2
:20012000590200085902000859020008590200080000fdff02001201100102000020fefff2
:020000040800f2
:200140000a0000010102030109024300020100c032090400000102020100052400100105f8
:020000040800f2
:2001600024010101042402020524060001070581030800ff09040100020a0000000705043b
:020000040800f2
:20018000024000000705850240000004030904200361006c007400750073006d00650074a4
:020000040800f2
:2001a00000720075006d002e006f0072006700160341006c0074006f00730046006c006146
:020000040800f2
:2001c00000730068000e03300030003000300030003100000000000008b500f055f828b13f
:020000040800f2
:2001e00000f082f810b1034800f03cf8024a034b9a6008bd001000080000000800ed00e01f
:020000040800f2
:2002000008b500f0a5f800f0a3fc00f06cfd002008bd000008b50a4a0a490b4800f00cfe16
:020000040800f2
:2002200000210a4a0a4800f015fe0a4800f042fe00f018fe00210846fff7e2fffee700bf82
:020000040800f2
:20024000680000005a0f00080c000020d4000000740000207400002070470e2008b500f00b
:020000040800f2
:200260003efd00004368074903f17842a2f580728a4205d8da0703d5026895469e467047cf
:020000040800f2
:20028000704700bf00ff1f0008b50a4b0a4a5968914203d19968094a914201d0012008bd1e
:020000040800f2
:2002a00000221868c3e901220028f8d0fff7dafff4e700bf00000020a5a55a5a3c3cc3c358
:020000040800f2
:2002c000044b054a05491860c3e90112044b054ada607047000000203c3cc3c3a5a55a5a50
:020000040800f2
:2002e00000ed00e00400fa054021144bda6942f08052da619a6942f008029a61104a1161e6
:020000040800f2
:20030000116821f0706141f000611160642100bf013989b20029fad190681168c0f380101e
:020000040800f2
:2003200021f0706141f0806111609a6922f008029a61da6922f08052da61704700100240d3
:020000040800f2
:20034000000c014030bf62b672b60020704770473a4b1a6842f001021a601a68920761d58c
:020000040800f2
:200360005a6822f003025a605a6812f00c025bd19a601a6822f480221a601a6842f48032d4
:020000040800f2
:200380001a601a68900351d512212d4a1160da6942f08052da615a6822f0f0025a605a68c9
:020000040800f2
:2003a00012f0f00f44d15a6822f4e06242f480625a605a6822f460525a605a6822f440429d
:020000040800f2
:2003c00042f400425a601a6822f080721a601a6891012fd45a6822f47c1242f4f8125a6074
:020000040800f2
:2003e0001a6842f080721a601a68920124d55a6822f0030242f002025a605a6802f00c0244
:020000040800f2
:20040000082afad15a6a42f080725a629a6942f001029a610b4a536823f0e06343f00073fc
:020000040800f2
:200420005360704700bf98e700bf9de700bfa8e700bfb4e700bfcae700bfd5e700100240ec
:020000040800f2
:20044000002002400000014070b572b60c4e049d56f8204041ea422104f4804284ea051533
:020000040800f2
:20046000114304f0400284ea0334114304f4405405f030052143294346f8201062b670bdc0
:020000040800f2
:20048000005c0040044b1a78012a9fbf511c19709b185870704700bf7400002030b50024d2
:020000040800f2
:2004a000a3b2d51aadb2012d10d85308c3ebc33402eb440292b242b110f8132051f8230072
:020000040800f2
:2004c00000f47f40024341f8232030bd055b5b0841f823500234e3e7002370b5461c9cb254
:020000040800f2
:2004e000151badb2012d0bd85308c3ebc33402eb440292b21ab151f8232000f8132070bd36
:020000040800f2
:20050000640851f82440c454c4f30724f4540233e5e738b5104d6b68e868dc682b7ac4f372
:020000040800f2
:2005200009049c4228bf1c461b1b2b721cb122462969fff7d1ff2044e86072b6074a136887
:020000040800f2
:2005400023f40f639b049b0c83f4304383f08003136062b638bd00bf74000020005c00407d
:020000040800f2
:2005600038b5124c04f11405237ddbb90123657da169402d237501d023771db12a460c48dc
:020000040800f2
:20058000fff78cff63680b4a5d6300236375d36823f0c0035b055b0d83f4004383f0b00346
:020000040800f2
:2005a000d36038bd2846fff7cdfedde77400002091000020005c0040164b70b51b6803f043
:020000040800f2
:2005c0003003302b24d0144c2378266e1f2b96bf1d4620250022a3eb050398bf84f85d20bb
:020000040800f2
:2005e000237025b12a463046616efff757ff63682e4426665d6072b6064a136823f0c00342
:020000040800f2
:200600005b055b0d83f4004383f0b003136062b670bd00bf005c0040740000202de9f74f2f
:020000040800f2
:200620000025ae4c10f00107064684f8685037d04022ab4b29461d65aa4b284663601a6023
:020000040800f2
:2006400003f180025d60626660229a604ff40042c03343f8b42c23618023a4f86a3002230e
:020000040800f2
:20066000012200930323fff7effe00233846012219460095fff7e8fe0130c7b2082ff4d181
:020000040800f2
:200680008022974bda6484f86c5084f86d5084f85d5025662570e560257203b0bde8f08f2b
:020000040800f2
:2006a00081072dd504f16e03e36008232372fff730ff237a23bb94f96e2094f86e30002a38
:020000040800f2
:2006c00046dbb4f87420002a0cbf0122022284f85d20854a13f0600022664ff000022270f7
:020000040800f2
:2006e00038d0202800f0e98094f85d30012b07d1b4f8743022789a4288bf2370fff75cff43
:020000040800f2
:2007000072070fd594f85d30022b0bd1fff701ff237a3bb9012284f85d20227802b12370d7
:020000040800f2
:20072000fff74aff3307b8d594f86c3043b194f876306b4a43f08003d364002384f86c3088
:020000040800f2
:2007400094f85d30012ba8d103b0bde8f04f33e70122bce703f01f03012b00f09c80022bea
:020000040800f2
:2007600000f0a080002bbfd194f86f30092bbbd801a252f823f000bfaf080008e906000847
:020000040800f2
:20078000e9060008e9060008e9060008a1070008b1070008e9060008eb070008f107000813
:020000040800f2
:2007a000b4f8703084f87630012384f86c309be7b4f870304d491d0a2f46dbb20a78002a56
:020000040800f2
:2007c00092d04878b8420ed1581ec0b253b9022d08bf8a78b4f874302166934238bfdab203
:020000040800f2
:2007e000227081e703461144e8e794f8770061e000254ff0020b0121d4f80480b4f86a70e5
:020000040800f2
:20080000b4f87030c8f8107084f8773008462b46c8f814500322cdf800b0fff715fe4ff460
:020000040800f2
:200820000443dff8c0a007f108091ffa89f9c8f82890c8f82c300aeb490307f14809a3676e
:020000040800f2
:200840002a4658461ffa89f9032304210095fff7fbfd88370aeb4903c8f83090a3612a462d
:020000040800f2
:200860002b460521c8f83450a4f86a700320cdf800b0fff7e9fd1e4825772575fff767fdbd
:020000040800f2
:2008800001231c4884f87c5084f8775084f86d30fff75dfd28e794f86f3043b10a2b7ff406
:020000040800f2
:2008a00023af07e094f86f30002b7ff41daf0020fff7e8fdfff7e6fd16e794f86f30202ba3
:020000040800f2
:2008c00007d0212b7ff410af0b4b2366072323700ae7094be3600723237205e77400002060
:020000040800f2
:2008e000005c004000600040750000203601000888000020e10000200c0000203b494b6cd8
:020000040800f2
:2009000018045fd540f20f7003f00f0351f82320104041f82300032b67d8dfe803f0023937
:020000040800f2
:200920001f2c334bb3f87e100131a3f87e10110409d593f8681010054cbf41f0020141f0df
:020000040800f2
:20094000040183f86810120642bf93f8682042f0080283f8682093f868005fe62448b0f8e8
:020000040800f2
:2009600080300133a0f8803013043ed5012300f87c3ffff7ecbc1e481106b0f8823003f1e1
:020000040800f2
:200980000103a0f8823030d5002300f8143ff0e717491206b1f8843003f10103a1f88430a5
:020000040800f2
:2009a00023d512494a6882f0200322f0f002520503f03003520d134343f4004343f0800337
:020000040800f2
:2009c0004b6070475b0510d5094bb3f886200132a3f886204a6c22f480624a6493f8680008
:020000040800f2
:2009e00040f0010083f86800b7e77047005c004074000020024a536c23f4805353647047fb
:020000040800f2
:200a0000005c004010b5064c94f86d301bb172b6237f0bb162b610bdfff7a2fdf8e700bf90
:020000040800f2
:200a20007400002070b50f4c054694f86d308bb172b604f11406627d3f2a0fd800232377cf
:020000040800f2
:200a4000531cdbb26375402b1444657701d1fff787fd62b670bd3046fff774fc237d002beb
:020000040800f2
:200a6000f9d1e8e774000020f8b572b61a4c04f18a0694f86d301bb30027184d94f88830c2
:020000040800f2
:200a800094f889209a421fd194f87c30c3b1636884f87c70da6ad2b284f889201ab1304648
:020000040800f2
:200aa000a16ffff719fd84f88870ab6823f40f639b049b0c83f4304383f08003ab60dde715
:020000040800f2
:200ac0000748fff73ffcd4e75a1c84f888201c4494f88a0062b6f8bd74000020005c0040ce
:020000040800f2
:200ae000f00000204ff080731449154a0b61d36943f40003d36172b6124a0120d2f814332c
:020000040800f2
:200b000023f0ff0343f0c003c2f814334ff48013136000220c4b83f877200c4b18641a64a4
:020000040800f2
:200b20005a644ff404421a6462b64ff47a7300bf013bfcd14ff480730b617047000801403e
:020000040800f2
:200b40000010024000e100e074000020005c00400d4a10b5936949f6404443f00403936149
:020000040800f2
:200b60004ff08073094a1361536823f00f0343f00103536000bf013cfcd1fff7b3ff044bf2
:020000040800f2
:200b800083f85d4010bd00bf00100240000801407400002008b5084b1a6912060ad5074aa7
:020000040800f2
:200ba0005a6002f188325a601b691b0602d5092000f095f808bd00bf00200240230167453c
:020000040800f2
:200bc0000d4b10b51b8804469bb2802b8cbf4ff400634ff48063013b18420bd172b6fff76c
:020000040800f2
:200be000d9ff204600f070f9044a136943f08003136162b610bd00bfe0f7ff1f002002406f
:020000040800f2
:200c000038b504460d46fff7dbff72b6fff7c2ff80222946204600f05bf9034a136943f0e4
:020000040800f2
:200c20008003136162b638bd0020024070b505460e461446fff7c4ff72b6fff7abff621c31
:020000040800f2
:200c400031462846520800f043f9034a136943f08003136162b670bd0020024070b5044620
:020000040800f2
:200c6000451814f8016b4eb10a2e02d10d20fff7d9fe3046fff7d6fea542f2d170bd38b597
:020000040800f2
:200c800005461c2425fa04f303f00f030a2b88bf273303f13000043cfff7c4fe231df1d1ba
:020000040800f2
:200ca00038bd10b5fff7e0fe2028fbd00024a0f13003092b05d9a0f16103052b06d8a0f105
:020000040800f2
:200cc000570343ea0414fff7cffef0e7a0f14103052b02d8a0f13703f3e7204610bdfee73f
:020000040800f2
:200ce0004ff6ff71bae780b5474d484e484fc0b0fff788fefff7b8fe58285bd027d85228ec
:020000040800f2
:200d00005dd05728f4d1fff7ccffea4604464ff48079d046fff7a8fe09f1ff391ffa89f96c
:020000040800f2
:200d20000af8010bb9f1000ff4d13a4b9c42dfd9394b1b889bb29b0203f10063a3f5807319
:020000040800f2
:200d40009c42d5d841462046fff75affd0e761282cd07628ccd13046fff7c2ff3846fff7b4
:020000040800f2
:200d6000bfff2e48fff7bcff2d48fff7b9ff2d48fff7b6ff2c48fff7b3ff2846fff77fff4d
:020000040800f2
:200d80002020fff74ffe244b188880b2800200f10060fff774ff2548fff7a2ff08212448ba
:020000040800f2
:200da000fff75cff2348fff79bffa1e72846fff787fa9de7fff775fffff702ff98e7fff720
:020000040800f2
:200dc00070ff144b0446984213d9134b1b889bb29b0203f10063a3f58073984209d800f5b8
:020000040800f2
:200de0008078234601341878fff71cfea045f8d17ee74ff48074013cff20a4b2fff712febb
:020000040800f2
:200e0000002cf8d174e700bf00100008ff0e00080c0f0008ff0f0008e0f7ff1fe70e00086b
:020000040800f2
:200e20001f0f0008dc0e0008320f0008450f0008f70e0008580f00080a44914200f1ff3325
:020000040800f2
:200e400000d1704710b511f8014b914203f8014ff9d110bd03460244934200d1704703f854
:020000040800f2
:200e6000011bf9e770b500260d4d0e4c641ba410a6420bd10c4b0bb1aff3008000260b4dcd
:020000040800f2
:200e80000b4c641ba410a64205d170bd55f8043b98470136ece755f8043b98470136f2e7ed
:020000040800f2
:200ea000d80e0008d80e000800000000d80e0008dc0e0008024bc01a024b1860704700bf14
:020000040800f2
:200ec00008000000400100205ff800f0190000205ff800f041000020d9010008416c746f0f
:020000040800f2
:200ee00073466c61736800616c7475736d657472756d2e6f726700312e392e3138000061c8
:020000040800f2
:200f00006c746f732d6c6f61646572000a6d616e7566616374757265722020202020000aaa
:020000040800f2
:200f200070726f6475637420202020202020202020000a666c6173682d72616e67652020de
:020000040800f2
:200f400020202020000a736f6674776172652d76657273696f6e20000a0000c2010000007c
:020000040800f2
:200f6000080000000000084b1a6942f002021a6158611a6942f040021a61da68d207fcd4cc
:020000040800f2
:200f80001a6922f002021a617047002002400b4b30b51c6944f001041c610024e5b2aa4207
:020000040800f2
:200fa00004d81a6922f001021a6130bd31f8145020f81450dd68ed07fcd40134eee7002019
:020000040800f2
:200fc00002400000ffffffffffffffffffffffffffffffffffffffffffffffffffffffffeb
:020000040800f2
:200fe000ffffffffffffffffffffffffffffffffffffffffffffffffffffffffffffffff11
:020000040800f2
:2010000000500020651200082d1300082f1300082f1300082f1300082f1300080000000071
:020000040800f2
:201020000000000000000000000000002d1300082d130008000000002d1300085127000858
:020000040800f2
:201040002d1300082d1300082d1300082d1300082d1300082d130008515400085554000882
:020000040800f2
:20106000595400085d54000861540008612b0008652b0008692b00086d2b0008712b000839
:020000040800f2
:20108000752b0008792b00082d1300082d130008915100082d1300082d1300086554000831
:020000040800f2
:2010a0002d1300082d1300082d1300082d1300082d1300082d1300082d13000805330008f8
:020000040800f2
:2010c0000d33000809330008113300082d1300082d1300082d1300082d1300082d130008d0
:020000040800f2
:2010e0006f5400082d130008915200082d1300082d1300082d1300082d1300082d1300088a
:020000040800f2
:201100002d1300082d1300082d1300082d1300082d1300082d1300082d1300082d1300088f
:020000040800f2
:201120002d1300082d1300082d1300082d1300080000fdff02001201100102000020feff4e
:020000040800f2
:20114000280000010102030109024300020100c032090400000102020100052400100105ca
:020000040800f2
:2011600024010101042402020524060001070581030800ff09040100020a0000000705042b
:020000040800f2
:20118000024000000705850240000004030904200361006c007400750073006d0065007494
:020000040800f2
:2011a00000720075006d002e006f00720067001c0345006100730079004d0065006700613a
:020000040800f2
:2011c000002d00760033002e0030000e03300030003000300030003100000000014a024b11
:020000040800f2
:2011e0009a6070470010000800ed00e008b500f0a3f800f08fff01f085f94ff4c06001f0d0
:020000040800f2
:2012000041f901f0e5fa02f0bbf901f0b5ff01f079fd04f04dfa03f029f903f0fbf900f0eb
:020000040800f2
:2012200059fb02f007fc02f0a5fd02f02dff03f047f803f049fb05f05ffc04f0b5fd04f060
:020000040800f2
:2012400091fb04f08df801f059fc05f031fd06f0dbf800f007ff4ff4c06001f023f901f000
:020000040800f2
:20126000fbf8000008b50a4a0a490b4806f090fd00210a4a0a4806f0b3fd0a4806f0e8fda7
:020000040800f2
:2012800006f0befd00210846fff7b0fffee700bf1c0000000cc000080c0000201027000092
:020000040800f2
:2012a00028000020280000204368074903f17842a2f580728a4205d8da0703d502689546c5
:020000040800f2
:2012c0009e467047704700bf00ff1f0008b50a4b0a4a5968914203d19968094a914201d019
:020000040800f2
:2012e000012008bd00221868c3e901220028f8d0fff7dafff4e700bf00000020a5a55a5a20
:020000040800f2
:201300003c3cc3c3044b054a05491860c3e90112044b054ada607047000000203c3cc3c3ff
:020000040800f2
:20132000a5a55a5a00ed00e00400fa0570470e2008b501f0a1f900003f4b1a6842f0010271
:020000040800f2
:201340001a601a68910768d55a6822f003025a605a6812f00c0262d19a601a6822f48022f0
:020000040800f2
:201360001a601a6842f480321a601a68920358d51a6842f001021a601a68900753d5122126
:020000040800f2
:201380002e4a1160da6942f08052da615a6822f0f0025a605a6812f0f00f46d15a6822f4b0
:020000040800f2
:2013a000e06242f480625a605a6822f460525a605a6822f4404242f400425a601a6822f0b5
:020000040800f2
:2013c00080721a601a68910131d45a6822f47c1242f4f8125a601a6842f080721a601a6886
:020000040800f2
:2013e000920126d55a6822f0030242f002025a605a6802f00c02082afad15a6a42f08072ef
:020000040800f2
:201400005a629a6942f001029a610d4a536823f0e06343f000735360704700bf91e700bf6f
:020000040800f2
:2014200096e700bfa1e700bfa6e700bfb2e700bfc8e700bfd3e700bf0010024000200240ea
:020000040800f2
:201440000000014008b501f0cff8bde808400020fff758bf1fb50e4b0e4a1b880e499bb2f0
:020000040800f2
:201460009b02a3f5805303930c4b0d481b680293182301930b4b1b8800930b4b1b8806f0c0
:020000040800f2
:20148000f1fc0a490a4805b05df804eb06f0eabce0f7ff1fe0a20008eea200084019002095
:020000040800f2
:2014a00006a30008941c002030110008fea20008a1a30008092894bf30305730c0b201f0a0
:020000040800f2
:2014c00081b810b5044614f8010b00b910bd01f079f8f8e72de9f8430025164f97f840201b
:020000040800f2
:2014e000ebb29a4201d8bde8f883002657f82380f3b208ebc30258f833300bb90135ede784
:020000040800f2
:2015000054682046fff7ddff204606f071fc431c04eb0309c0f12d043cb94846fff7d1ff89
:020000040800f2
:201520000a2001f04ff80136e2e7202001f04af8013cf1e72800002070b5044601f078f8a9
:020000040800f2
:2015400010b12046fff7bdff00232e4c2e4e84f8413001f049f801f054f81528054623d0c2
:020000040800f2
:2015600015d80a2825d00d2823d0082894f8413037d1002bedd001f05bf810b12248fff7ad
:020000040800f2
:20158000a0ff94f84130013b84f84130e1e77f28ece701f04df810b13046fff792ff94f8c4
:020000040800f2
:2015a0004130013b84f8413094f84130002bf0d1cfe701f03df810b10a2001f003f80a21ca
:020000040800f2
:2015c00094f84130e21882f842109a1c84f8412000220133dbb2234483f8422084f8c22030
:020000040800f2
:2015e00070bd7d2bb5d85a1c234484f8412083f8425001f01df80028abd0284600f0e2ffda
:020000040800f2
:20160000a7e700bf28000020dcaa00080a220a4b93f8411083f8c32093f8c220914207d9cc
:020000040800f2
:20162000511c1a4492f8422083f8c21083f8c32093f8c300704700bf2800002008b500f08f
:020000040800f2
:20164000e0ff03463038c0b2092806d9a3f16102d2b2052a02d8573bd8b208bda3f141023c
:020000040800f2
:20166000d2b2052a01d8373bf6e70122024b002083f8c420f1e700bf2800002010b50446b2
:020000040800f2
:201680000009fff717ff04f00f00bde8104011e710b50446000afff7f1ffe0b2bde81040bf
:020000040800f2
:2016a000fff7ecbf054b93f8c300202804d0a0f10903584258417047012070472800002028
:020000040800f2
:2016c00008b5fff7efff00b908bdfff79ffff8e7f8b51d4e1d4c3046fff72efffff796ffd3
:020000040800f2
:2016e000fff7eeff94f8c350fff790ff0d2df2d00a2df0d0002394f840c01448dab2944580
:020000040800f2
:2017000003d8022384f8c43017e0002250f8047bd1b207ebc10e57f8311009b90133ede7db
:020000040800f2
:20172000def804e001329ef800e0ae45f0d1884794f8c430013b012bcdd80548fff7c1fe34
:020000040800f2
:20174000002384f8c430c6e749a9000828000020b8a30008a0f13003dbb2092b01d858b23c
:020000040800f2
:201760007047a0f16103052b02d8573840b27047a0f14103052b01d83738f7e74ff0ff30e2
:020000040800f2
:201780007047f8b5002405462646fff799ff0c4f97f8c300fff7deff002808dae4b20cb19f
:020000040800f2
:2017a000ff2d02d0012387f8c4303046f8bd013440ea0616fff72affac42e9d1f5e700bf8c
:020000040800f2
:2017c0002800002008b50220fff7dbffc0b208bdff20d6e708b5fff7fbff074b93f8c43081
:020000040800f2
:2017e00043b9003818bf0120044b1a78044b03eb0213187308bd00bf2800002015050020f9
:020000040800f2
:2018000004050020f8b5114dfff75aff95f8c3302d2b11d1fff7fafe0126012200240a27fe
:020000040800f2
:2018200095f8c330303bd9b2092907d807fb0434fff7ecfe0022f3e70026eee712b1012329
:020000040800f2
:2018400085f8c43006b164422046f8bd2800002038b5094d441e14f8013f0bb9012007e09a
:020000040800f2
:2018600095f8c3209a4204d00223002085f8c43038bdfff7cbfeeee72800002008b5fff70e
:020000040800f2
:201880001fff0848fff7e4ff50b100f0adfe642000f07afd044b054a0820da6000f0ecfea0
:020000040800f2
:2018a00008bd00bfc6a3000800ed00e00400fa0508b5074b93f840200f2a02d9062000f03f
:020000040800f2
:2018c000dbfe511c83f8401043f8220008bd00bf2800002008b50548fff7eaffbde80840f8
:020000040800f2
:2018e000034a0449044800f029bc00bfe0aa0008cca30008d1160008f000002010b503f0ae
:020000040800f2
:2019000034f9094c094b2068196802f097ff4ff480720749206802f02dff002004f074f8b5
:020000040800f2
:20192000bde8104003f020b9401900203c190020180300202de9f04100254ff00c080a4ea6
:020000040800f2
:201940000a4febb208fb03f3f45801350cb9bde8f081204606f04cfa421c214638462244f0
:020000040800f2
:2019600006f080faede700bf70ab0008d0a30008024b034893f8fc1006f074ba1803002038
:020000040800f2
:20198000daa30008024b034893f8f81006f06aba18030020eea30008024b0348b3f8fa105c
:020000040800f2
:2019a00006f060ba1803002002a40008024b0348197f06f057ba00bf1803002011a4000840
:020000040800f2
:2019c000034b0448996941f38f2106f04bba00bf1803002022a40008024b0348597f06f05e
:020000040800f2
:2019e00041ba00bf1803002039a4000810b5094c0948b4f91220b4f9041006f033fab4f932
:020000040800f2
:201a0000f630b4f9f420b4f9f2100448bde8104006f028ba180300204ea4000869a40008cd
:020000040800f2
:201a2000024b0348998f06f01dba00bf1803002090a40008024b0348197c06f013ba00bf34
:020000040800f2
:201a400018030020aca40008024b0348598806f009ba00bf18030020c6a400082de9f74ff9
:020000040800f2
:201a6000002501462b4806f0fdf900f0bdfd00f0c8fd294806f00efa00f0b6fd274806f0c5
:020000040800f2
:201a800009fa2e4600f0b0fd2f46a9464ff48062dff88ca0dff88cb09af800105046cde9a5
:020000040800f2
:201aa000002100f0cffb0199009a0b4690461c469af800c0194642460beb831008f1ff389c
:020000040800f2
:201ac0000133a44503f01f031ffa88f8e6d0009301f0bcfd0beb8414a28e009b12b21744d0
:020000040800f2
:201ae000e28e814412b2b61a228f12b21544b8f1000fdcd10c4bbf12b612ad1249f38f2050
:020000040800f2
:201b0000a3f80071a3f80261a3f8045103b0bde8f08f00bfdea4000803a5000806a5000848
:020000040800f2
:201b2000ec1f0020a40700201803002070b5fff7c7fd0c4b0c241d78fff768fd00220a49a9
:020000040800f2
:201b4000d3b26343c818cb581bb90222074b1a7070bd1b780132ab42f2d14368bde87040e0
:020000040800f2
:201b6000184700bfeb00002070ab0008ec00002038b50c4d05f5837000f051fe95f80741c6
:020000040800f2
:201b80002cb1fff7bbfe0023012485f80731064800f062fe24b10548bde8384006f07ab9b6
:020000040800f2
:201ba0000348f9e7180300201e04002015a500081ba5000810b5054c204600f030fefff763
:020000040800f2
:201bc0009dfe2046bde8104000f046be1e04002038b5434c04f5837000f021fe94f808517d
:020000040800f2
:201be000002d7bd102f0c1ff3e4b4ff480721868214602f049fd2378012b0ed023463a4a4b
:020000040800f2
:201c0000a4f80d5043f80d2b9d70384ba5711a689b88c4f80720a4f80b3065781a2d5ad005
:020000040800f2
:201c200005f076fb9db925740023a38063824ff48013a3610023237700236377012384f8f0
:020000040800f2
:201c40002430102200212a4806f0caf80be0012dead0032debd9042decd0052decd0072ddd
:020000040800f2
:201c6000ecd9082dedd0092d22d86422a379534303f5d42303f5bb73a3630023a387b0220b
:020000040800f2
:201c800000211c4806f0acf80023a4f8f0300023a4f8f230c4f8f430a38063825e2384f880
:020000040800f2
:201ca000f8300523a4f8fa30002384f8fc300de00a2de2d00b2de2d00c2de5d00e2de6d99b
:020000040800f2
:201cc0000f2debd0112decd9192dedd91a236370012384f80731012384f8083138bd00bf89
:020000040800f2
:201ce00018030020401900200100fa002ba500083d030020580300200123034880f8073163
:020000040800f2
:201d000000f5837000f0a8bd1803002010b5fff779fd084b04461b785bb9fff759ff003c4c
:020000040800f2
:201d200018bf0124044b83f8fc40bde81040fff7e3bf10bdec0000201803002010b5fff745
:020000040800f2
:201d400061fd074b04461b7843b9fff741ff054b83f8f840bde81040fff7cebf10bd00bfbd
:020000040800f2
:201d6000ec0000201803002010b5fff74bfd074b04461b7843b9fff72bff054ba3f8fa40a9
:020000040800f2
:201d8000bde81040fff7b8bf10bd00bfec0000201803002010b5fff735fd064b04461b78f3
:020000040800f2
:201da0003bb9fff715ff044b1c77bde81040fff7a3bf10bdec0000201803002010b5fff727
:020000040800f2
:201dc00021fd134b1b7813bb840203f0ddff40b1104b9b69a3421ad0bde810400e4806f071
:020000040800f2
:201de00059b80e4b1968a14205d2bde810400c48890a06f037b8fff7ebfe0a4b054a1b6877
:020000040800f2
:201e00005b422340bde810409361fff775bf10bdec0000201803002032a500084019002043
:020000040800f2
:201e200061a500083c19002010b5fff7ebfc0c4b1b789bb900f00104fff7cafe094b5a7f5f
:020000040800f2
:201e4000a24206d0b3f90420598a5242494299805a825c77bde81040fff74ebf10bd00bfaa
:020000040800f2
:201e6000ec000020180300202de9f04fdff800a185b0fff7c7fc9af80030002b74d104b278
:020000040800f2
:201e8000fff7c0fc24bb9af800300bb339488af80040fff7e3fd384d04463848b5f900b16a
:020000040800f2
:201ea000b5f90281b5f90471fff7d8fdb5f90011b5f90221b5f9043106460125b44212db3b
:020000040800f2
:201ec000324621462e4805b0bde8f04f05f0cabf002506b22b462f462a46a8462946ab4615
:020000040800f2
:201ee0008af80050eae7dff89090cde902230191fff76efea9f80440a9f81260ddb1019959
:020000040800f2
:201f0000029a039b8b4490441f440bebdb7b08ebd87807ebd7774fea6b0b4fea68087f10cb
:020000040800f2
:201f2000a9f8f2b0a9f8f480a9f8f67005b0bde8f04ffff7e1befff765fc9af80030002bd0
:020000040800f2
:201f4000f4d1a9f8f200fff75dfc9af80030002becd1a9f8f400fff755fc9af80030002b67
:020000040800f2
:201f6000e4d1a9f8f600e1e705b0bde8f08f00bfec00002077a50008180300207aa5000823
:020000040800f2
:201f80007fa5000810b5fff73dfc094b04461a7822b9b0f5803f02d301221a7010bdfff76d
:020000040800f2
:201fa00017fe044b9c87bde81040fff7a5be00bfec0000201803002010b5fff723fc084b19
:020000040800f2
:201fc00004461a781ab9ff2802d901221a7010bdfff7fefd034b1c74bde81040fff78cbed2
:020000040800f2
:201fe000ec0000201803002010b5fff70bfc064b04461b783bb9fff7ebfd044b5c80bde808
:020000040800f2
:202000001040fff779be10bdec0000201803002008b5fff7ddfdbde80840014800f01cbca4
:020000040800f2
:202020001e04002070b5fff7f3ff0b4b0b485a78197805f017ff00240c26094de3b2734343
:020000040800f2
:20204000ea18eb581bb9bde8704001f0bdbc936803b198470134f1e718030020a1a5000884
:020000040800f2
:2020600070ab00080148fff723bc00bf24ac0008d0e9002353601a60c0e9000070470146d8
:020000040800f2
:2020800008b51430fff7f4ff034b5a685860c1e90532106008bd00bf2404002008b51c3068
:020000040800f2
:2020a000fff7e6ff054a134653f8081f99420cbf002351f8183c136108bd00bf2404002085
:020000040800f2
:2020c0002de9f843eff31088074672b64ff000090f4e56f8084f54f81c591c3d04f11c0348
:020000040800f2
:2020e000b34203d06368fb1a002b03da88f31088bde8f8832046c4f80490fff7cfff20461d
:020000040800f2
:20210000fff7bdffeb692c46a3f11c05e6e700bf24040020084b03f10802c3e9022200227b
:020000040800f2
:20212000c3e900331a6114330132102ac3e9003303f10803f8d1704724040020f8b5244dcd
:020000040800f2
:20214000044695f89470102f3fd1012000f094fa56f804cb01309cf808c09c4505d1013321
:020000040800f2
:2021600013f0ff0306d000201a4e5ffa80fc6745eed8f4d10026237222612660c4f824123a
:020000040800f2
:202180003422314604f5f87005f02afe04f5f473e36004f11403c4e9053304f11c03c4e99f
:020000040800f2
:2021a0007a66eff31086c4e9073372b62046fff766ff95f8943005eb83020133c2f898406b
:020000040800f2
:2021c00085f8943086f31088f8bd0123cbe700bf24040020bc040020194cd4f8d8305bb1f6
:020000040800f2
:2021e0002de9ff5feff3008001b4eff3108001b46b46d4f8d820d36072b6d4f8d80018b1f0
:020000040800f2
:2022000003680bb9fff73bff2368a34207d194f8dc3013b162b672b6f6e730bffae7a3f13a
:020000040800f2
:202220001402c4f8d82053f8083c9d4601bc80f3108801bc80f30088bde8ff5f704700bf69
:020000040800f2
:202240002404002070b5eff31085014672b6114cd4f8d860304640f8141bc1f38301fff7bf
:020000040800f2
:2022600007ff04ebc1039a69986104f1140303ebc103c6e90532106085f31088fff7acffe4
:020000040800f2
:20228000d4f8d8300022186810b10120c3e9002270bd00bf240400202de9f041144b0546f3
:020000040800f2
:2022a00093f89420b2b1eff31087c0f3830203f11406d10006ebc20672b64ff000080b4475
:020000040800f2
:2022c000586950f81449143c00f114039e4203d187f31088bde8f0810368ab4203d1c0f880
:020000040800f2
:2022e0000080fff7ccfe63692046a3f11404ebe7240400202de9f04106460f4661b3eff3c8
:020000040800f2
:20230000108872b600f008fa7d1c1e4a0544012d104638bf0125d2f8d84050f8083f6560ea
:020000040800f2
:202320001c3b03f11c01814204d104f11c01d368d16008e05968491b090421d41b6a04f196
:020000040800f2
:202340001c0118684160c4e907031960936853f8183c136188f310883046fff773ff0446c6
:020000040800f2
:202360005fb1eff3108572b6064bd3f8d80000234360fff793fe85f310882046bde8f081e1
:020000040800f2
:20238000db69cde7240400200128014638bf01210148fff7afbf00bf0105002080b572b685
:020000040800f2
:2023a000194c002504f198031e4694f89420d4f8d880efb2ba4205f101011ed808f11400a3
:020000040800f2
:2023c000fff756fe08f11c00fff752fe94f8943006eb8101013bdbb2da1bd2b29200bb42c4
:020000040800f2
:2023e00038bf002206eb850084f8943005f0defc0023c4f8d830fff7effe53f8040b404596
:020000040800f2
:20240000dcd00d46d5e700bf24040020f7b500f083f9002405460e4e0e4f96f89420e3b2e3
:020000040800f2
:202420009a4201d803b0f0bd06eb8303d3f89800017ad0e9002343b15b1b1bb20069013481
:020000040800f2
:202440000090384605f00efde7e742f20f73f5e724040020b8a50008002208b5084bc3f874
:020000040800f2
:20246000d820eff3088383f30988eff3148343f0020383f31488bff36f8ffff7adfe00bf1d
:020000040800f2
:2024800024040020c20742bf4ff40072044b1a61830742bf4ff48062014b1a61704700bfbe
:020000040800f2
:2024a00000080140c20742bf4ff00072044b1a61830742bf4ff08062014b1a61704700bfa5
:020000040800f2
:2024c0000008014000f0010383f001025b0243ea4263054ac0f34000136180f0010380026e
:020000040800f2
:2024e00040ea8360106170470008014010b50446fff7c8ff0846fff747ff2046bde81040ad
:020000040800f2
:20250000fff7d0bf2de9f0430024012603272648dff898c0dff898e002680379624524d10a
:020000040800f2
:20252000244da96941f00401a961dd0803f110019b0003f01c0306fa01f11161991c52f8de
:020000040800f2
:20254000258007fa03f907fa01f141ea090128ea010806fa03f343ea080342f825300830a1
:020000040800f2
:202560000cb1bde8f0830124d6e7724504d1114da96941f00801d7e70f498a4204d10d4d5d
:020000040800f2
:20258000a96941f01001cfe70c498a4204d1094da96941f02001c7e709498a42c5d1054dcd
:020000040800f2
:2025a000a96941f04001bfe728ae000800080140000c014000100240001001400014014085
:020000040800f2
:2025c000001801400a2838b50446054d02d10d206b68984720466b689847002038bd00bf49
:020000040800f2
:2025e00004050020fff7eebf024b9b6803b11847704700bf0405002008b5fff7f5ff002046
:020000040800f2
:2026000008bd38b572b6074c04f1100523689847431c03d12846fff715fef7e762b6c0b207
:020000040800f2
:2026200038bd00bf0405002008b5fff7eaff08bd014b187b704700bf04050020034b9a6096
:020000040800f2
:202640000122c3e900011a7300207047040500200138c0b2ff2308e000bf013a12f0ff026b
:020000040800f2
:20266000fad1013b13f0ff0301d0ff22f4e70138c0b2ff28eed1704708b572b600f040061e
:020000040800f2
:2026800000f03f051420fff7e3ff05244b2001f083ff0120fff7dcff962001f07dff013ca1
:020000040800f2
:2026a0000120fff7d5ff14f0ff04efd1204601f073ff0220fff7ccff9eb14ff40070fff7c4
:020000040800f2
:2026c000e1fe4b2001f068ff2820fff7c1ff4ff40070fff7e7fe204601f05eff0a20fff7f8
:020000040800f2
:2026e000b7ff0024e3b29d42ccd94ff40070fff7c9fe5e2001f050ff0a20fff7a9ff4ff4ae
:020000040800f2
:202700000070fff7cffe002001f046ff0a20fff79fff0134e6e70000014b1868704700bf2e
:020000040800f2
:202720001805002010b5074a074c1368a06811688b42fad16f21a0fb0101044ae3fb020103
:020000040800f2
:2027400010bd00bf1805002010e000e080969800124b10b51b68db031fd5114c114a236878
:020000040800f2
:2027600012680133236023689b1a002b02db2068fff7a6fc23790c4a0133dbb223711178f0
:020000040800f2
:202780008b420ad1137843b10023237101f03cfebde810400548fff77fbd10bd10e000e01f
:020000040800f2
:2027a00018050020340400201c0000201c050020eff3108372b60021034a1070034a1171ad
:020000040800f2
:2027c00083f31088704700bf1c00002018050020064b074a5a6000229a6003221a60054a96
:020000040800f2
:2027e000136a43f070431362704700bf10e000e08f5f010000ed00e008b503788b4202d127
:020000040800f2
:202800000320fff739ffeff3108372b6027822b90170012083f3108808bd0020fae770b5ea
:020000040800f2
:202820000c4d02782b6804461b7a9a4202d10320fff722ffeff3108672b623782bb92b68b8
:020000040800f2
:202840001b7a237086f3108870bd2046fff7fafcf3e700bffc04002010b5094a01781268fc
:020000040800f2
:20286000127a914202d00320fff706ffeff3108472b600220270fff70ffd84f3108810bdf9
:020000040800f2
:20288000fc0400202de9f0411b4e00eb400333445a7804460d464fea400852bb01229042d1
:020000040800f2
:2028a000164f9a705a701cd049b1154a137c33b1127f022a03d064205843fff765fd0123fc
:020000040800f2
:2028c00005203b61fff760fd4ff480333b610023a0444644b37065b1bde8f041c820fff7d4
:020000040800f2
:2028e00053bd022305203b61fff74efd4ff40033ece7bde8f08100bf2005002000080140f5
:020000040800f2
:202900001803002008b5fff783fb1c4c1c4d2046fff798fc2b7f032bf9d8dfe803f0021213
:020000040800f2
:202920001b1f2378063b012bf1d801210020fff7a9ff2378072bead101210846fff7a2ff1d
:020000040800f2
:20294000e5e72378063b012be1d801210020fff799fff1e72378072bd9d1f6e72378043b14
:020000040800f2
:20296000032b03d801210846fff78cff2378063b012bccd801210020e0e700bf5020002059
:020000040800f2
:202980001803002010b5fef79bfe1748fef760ff40b3164cfef794fe23786d2b0ad11448b0
:020000040800f2
:2029a000fef756ff30b100210120124b1971bde8104067e72378642b08d10f48fef748ffea
:020000040800f2
:2029c00020b100210b4b08465970f0e720783038c0b2092803d8bde8104004f083bc0222f7
:020000040800f2
:2029e000064b1a7010bd00bfd6a50008eb000020dba5000820050020e0a50008ec0000207c
:020000040800f2
:202a000030b5eff31085044691b072b6684600f005fe174904eb44028b18895c5a7885f39f
:020000040800f2
:202a200010889b78fbb901b1eab1b4b1012c17d040f2cd1040f2e932bdf91230934214dd57
:020000040800f2
:202a4000b0ebe30f11dbc3eb031343f30f139842d4bf0020012011b030bdbdf90c00e9e7f3
:020000040800f2
:202a6000bdf90e00e6e70220f5e70320f3e700bf2005002038b50020fff7c2ff0a4d0b4c54
:020000040800f2
:202a800055f820200a49204605f0ecf90120fff7b7ff084955f82020204605f0e3f9bde88f
:020000040800f2
:202aa000384004f0e0ba00bf3cae0008e7a50008e0a50008dba500084ff480320d498b6977
:020000040800f2
:202ac00043f004038b610c4b1a611a6822f00f0242f001021a608a6942f004028a614ff451
:020000040800f2
:202ae00000321a611a6822f0f00242f010021a60704700bf001002400008014008b5fff721
:020000040800f2
:202b0000dbff0548054a0649fff718fbbde808400448fef7cdbe00bf2805002000a6000874
:020000040800f2
:202b2000052900084cae00080f220b4930b40c688500aa4022404a60084a034652f82010f0
:020000040800f2
:202b400009b130bc084711180120087702f11c00184430bcfff7a0bb000002405007002056
:020000040800f2
:202b60000020e1e70120dfe70220dde70320dbe70420d9e70520d7e70620d5e708b50a4b00
:020000040800f2
:202b80001a1892f8231049b192f82a3013b10220fff772fdff2382f82a3008bd2a331844a9
:020000040800f2
:202ba000bde80840fff73bbe50070020064b1a1892f8231019b1002382f82a3070472a33ad
:020000040800f2
:202bc0001844fff749be00bf500700202de9f8431d4e99463318174693f82320054688463c
:020000040800f2
:202be0005ab393f82a2012b10220fff745fdff2283f82a20eff3108172b696f831305a1cf0
:020000040800f2
:202c000086f8312023b9114a536943f00103536181f3108814246c43089b04f1804404f5bf
:020000040800f2
:202c2000003443f00203a3600023c4e90487c4f80c9046f82530bde8f88306f12a00284432
:020000040800f2
:202c4000fff7edfdd6e700bf5007002000100240014b43f820107047500700200022074bf6
:020000040800f2
:202c600003441a771423584300f1804000f50030836843f001038360704700bf50070020e2
:020000040800f2
:202c80001423434303f1804303f500339a6810b4eff3108422f001029a6072b60e4b93f83e
:020000040800f2
:202ca0003120013ad2b283f8312022b90b494a6922f001024a6184f31088034493f8232072
:020000040800f2
:202cc00022b1002283f82a2010bc7047044b10bc1844fff7c1bd00bf500700200010024044
:020000040800f2
:202ce0007a07002008b5064b184490f8233013b10220fff7c1fc012380f8233008bd00bfe2
:020000040800f2
:202d0000500700202de9f0430b224ff001084ff0ff0e4ff0800c00270f48104cc61d08faa8
:020000040800f2
:202d200002f391102360c031d30054f8215003f018030efa03f925ea09050cfa03f301329b
:020000040800f2
:202d40002b43122a44f8213000f8017b06f8017be5d1bde8f08300bf7307002000e100e066
:020000040800f2
:202d6000012832d0042819d0002847d12022244b1a611a6822f4700242f480121a601a68d9
:020000040800f2
:202d800022f0706242f080621a6080221a611a6822f0704242f080521a6070470822194b9b
:020000040800f2
:202da0001a611a6822f4704242f480521a601a6822f4702242f480221a6020221a611a6811
:020000040800f2
:202dc00022f4700242f48012e6e74ff400520d4b1a615a6822f4700242f440125a605a6820
:020000040800f2
:202de00022f0706242f080625a604ff400421a615a6822f0704242f040525a60704700bfa7
:020000040800f2
:202e000000080140000c01402de9f041dff8d0800f4600f0010100f00d060446314b18f88e
:020000040800f2
:202e2000010003ebc103b0425d6820d0fff798ff012e41d0042e27d0beb92b4a536823f088
:020000040800f2
:202e400001035360294b1a6822f4700242f410021a601a6822f0706242f080621a601a6805
:020000040800f2
:202e600022f0704242f010421a6008f80160e10801f0020141eac701c4f34014214341f4bb
:020000040800f2
:202e800051712960bde8f081174a536843f001035360174b1a6822f4704242f410421a601d
:020000040800f2
:202ea0001a6822f4702242f480221a601a6822f4700242f41002d7e70d4b5a6822f47002e4
:020000040800f2
:202ec00042f430025a605a6822f0706242f080625a605a6822f0704242f030425a60c4e7cd
:020000040800f2
:202ee00082070020b0ae00080000014000080140000c014037b5094c04ebc00041f21004b5
:020000040800f2
:202f0000456844eac3144078134600940a4605f10c01fff75bfe03b030bd00bfb0ae0008f3
:020000040800f2
:202f200037b5094cdb0104ebc0056d6843f44053009314f8300013460a4605f10c01fff7b0
:020000040800f2
:202f400045fe03b030bd00bfb0ae00082de9f843eff31088154b03ebc00213f830400323ed
:020000040800f2
:202f60005568567820466b60fff778fe3046fff775fe72b60e4f04eb07093b5d8bb188f377
:020000040800f2
:202f80001088ab689b07fcd5ab6813f08003fbd130466b60fff774fe2046bde8f843fff7c9
:020000040800f2
:202fa0006fbe4846fff74ef9e7e700bfb0ae00086c07002038b50d4602f0010401230a46e8
:020000040800f2
:202fc00001462046fff796ff204600232a460349fff7a6ff2046bde83840b7e7840700200d
:020000040800f2
:202fe00037b50d4602f001048df807000a4620460df107010023fff77dff00232a462046c5
:020000040800f2
:203000000349fff78dff2046fff7a0ff03b030bd840700200022044b00f0010003ebc00389
:020000040800f2
:203020005b685a60704700bfb0ae0008084b00f0010003ebc0035b689a689207fcd59a6811
:020000040800f2
:2030400012f08002fbd1d96899685a60704700bfb0ae00080d4b02f0010203ebc203002226
:020000040800f2
:203060005b6801445a60884208d19a689107fcd59a681206fcd4da689b6870479a689207ff
:020000040800f2
:20308000fcd510f8012bda60ede700bfb0ae000870b5ff230d460646094902f00104204663
:020000040800f2
:2030a0002a4601f8023f0023fff724ff20462a4631460123fff734ff2046bde8704045e7a9
:020000040800f2
:2030c0008207002070b50d46164603f00104014601232046fff70eff204632462946012336
:020000040800f2
:2030e000fff71eff2046bde870402fe738b500f00103044606480d4618441146fff77cfb00
:020000040800f2
:2031000020b120462946fff77ffe012038bd00bf8507002038b504460d4600f0010304484b
:020000040800f2
:203120001844fff77cfb29462046bde838406be6850700200022054b00f0010003ebc003c3
:020000040800f2
:203140005b681a60024b1844fff786bbb0ae00088507002038b5074d00f001040146285d3e
:020000040800f2
:20316000fff7fefd0c232b550846bde83840fff7e1bf00bf82070020002070b50c26044685
:020000040800f2
:203180001349144d8b692e7043f004038b618b6943f008038b618b6943f480538b61fff7bc
:020000040800f2
:2031a000dffd0d4b18605860da689b688b69012043f008038b61cb696e7043f48043cb61ef
:020000040800f2
:2031c000fff7cefd054b1c605c60da689b6870bd0010024082070020003001400038004050
:020000040800f2
:2031e000f8b504461f4b204d03ebc0035e682b8877690133f8072b8042bf05eb44035b88fe
:020000040800f2
:203200003361b9070ad501227368184823f40073736020442b199a71fff73ef87a0707d584
:020000040800f2
:203220007368124823f4007373602044fff734f87b0616d505eb4402138961008bb105ebab
:020000040800f2
:203240008405eb6830695c1c18701389ec60013b9bb213812bb9bde8f84005480844fff7a4
:020000040800f2
:203260001bb8f8bdc0ae0008880700208e070020900700200a4b30b403ebc00359684a69d7
:020000040800f2
:2032800053050bd50225074b22f480621c18a57106334a61184430bcfef7febf30bc7047ba
:020000040800f2
:2032a000c0ae0008880700200021084b03ebc0035b685a69920705d501316429f9d10448f6
:020000040800f2
:2032c00004f0d0bd0029fad1704700bfc0ae000822a6000870b504466425084b03ebc003c1
:020000040800f2
:2032e0005e6833689b0503d5fef776ff013df8d10022034b23449a7170bd00bfc0ae000840
:020000040800f2
:203300008807002000206be7012069e70020b1e70120afe7064b10b503ebc0035c68054bd1
:020000040800f2
:203320001844fff77cfa00236361a36110bd00bfc0ae00089c070020014b1844fff78cba31
:020000040800f2
:203340009c070020f8b5184d184b2a18044603ebc0030020907105eb4402518024225b68c7
:020000040800f2
:203360005a6040f201121a6064221968c90501d5013afad172b64ff4497220465a60fff7e7
:020000040800f2
:203380002fff0b4e2f192644bb792bb919213046fef7b0ff0028f7d062b62544a879431e96
:020000040800f2
:2033a00058425841f8bd00bf88070020c0ae00088e0700202de9f04f14462c4a984602eb9c
:020000040800f2
:2033c000c4035d6885b08146204612f834700e4693f801a0ab69fff767ff41f290034a460b
:020000040800f2
:2033e00005f11001384600933346fff7effb5046fff7c4fb40f6240338466b60fff72efc4b
:020000040800f2
:2034000072b6dff86c90711c07eb090b19f8073033b958460391fef76dff03990028f5d0ce
:020000040800f2
:203420004ff449736b60134b013603eb04096b695b0705d431464846fef75cff0028f6d0e0
:020000040800f2
:2034400024236b6062b6b8f1000f05d040f2012320462b60fff73eff5046fff7a7fb38468f
:020000040800f2
:20346000fff70efc012005b0bde8f08fc0ae00086c0700208e0700202de9f74f8146144617
:020000040800f2
:2034800098460e46002971d0394a012902ebc4035d6833d1dff8dca067000aeb8403d860f8
:020000040800f2
:2034a0000aeb4403198120462960ab69fff7fcfe40f224736b60b8f1000f02d040f20123cf
:020000040800f2
:2034c0002b6072b62c4d0aeb07063d4433892bb101212846fef70eff0028f7d062b6574471
:020000040800f2
:2034e0003e89b6fa86f67609b8f1000f02d02046fff7f0fe304603b0bde8f08f12f834a05b
:020000040800f2
:203500005f785046fff73afb4ff402534a4605f11001384600933346fff758fb40f201439b
:020000040800f2
:203520002b6041f6240320466b60ab69fff7bcfe3846fff793fb72b6dff8409007eb090bd6
:020000040800f2
:2035400019f807302bb931465846fef7d3fe0028f6d062b640f20123384619f807602b6087
:020000040800f2
:20356000fff78efb5046fff721fbbde70126c1e7c0ae000888070020900700206c07002042
:020000040800f2
:20358000224b23499a6942f008029a614a6822f4706242f460624a609a6942f008029a61a2
:020000040800f2
:2035a0004a6822f4704242f460424a60da6942f48002da614ff40042164b1a60642200bf34
:020000040800f2
:2035c000013afcd124211a6059605969996919695a619a6148f224020421da610122196211
:020000040800f2
:2035e0001a6002220c4b5a60d3f8202322f47f4242f40042c3f820235960d3f8202322f4e4
:020000040800f2
:203600007f0242f40002c3f82023704700100240000c01400058004000e100e030b50a4b0a
:020000040800f2
:2036200013f8042b013a02f01f0203eb8213024603f140051c4603ccac4210605160234655
:020000040800f2
:2036400002f10802f6d130bda0070020034ac38d527f18b20ab95b4218b27047180300209e
:020000040800f2
:2036600008b501210020fff755fd4ff40022014b1a6108bd0008014008b50448062102f0a7
:020000040800f2
:203680000bf8bde808400248fef706be00080140a80f00207fb58df80700fff7e1ff06215a
:020000040800f2
:2036a0001c4801f0edff002201210df10700fff781fc0020fff74efd72b6164c164da368b4
:020000040800f2
:2036c0005b0605d401212846fef714fe0028f6d00621104801f0e0ff62b6082600252661ea
:020000040800f2
:2036e000fff7beff03a92b46084604228df80c50fff7e8fc28462661fff71cfd9df80e0024
:020000040800f2
:203700009df80d30b04040ea03409df80f30184304b070bd00080140a80f0020f7b53b4d16
:020000040800f2
:20372000ac7c002c50d11e2301268df80730ae74fff796ff314622460df10700fff73afc33
:020000040800f2
:203740003046fef721fe0823314e20463361fff7f1fcaf1c64f05f038df80730fff780ffa6
:020000040800f2
:20376000002201210df10700fff724fc381900220221fff78dfc0823002033610234fff7ca
:020000040800f2
:20378000d9fc102ce6d10023224a12f8011be9b90133102bf9d1204a137843f00203137021
:020000040800f2
:2037a0001e4a11780b43137008221d4b13f8021c13f8010c013a12f0ff0203f8020c03f832
:020000040800f2
:2037c000011c03f10203f1d103b0f0bd00231022104c687c6b7414f8011b4b4008211eb291
:020000040800f2
:2037e0005b00002e9bb201f1ff31b8bf83f4405311f0ff01f3d1013a12f0ff02ebd16874b5
:020000040800f2
:2038000000f00f00b0eb133fc5d1cde7a80f002000080140aa0f002052200020a40f002014
:020000040800f2
:20382000ac0f002010b504464620fff733ff20605620fff72fff606010bd83b5fff76effce
:020000040800f2
:203840000a4e0b4d0b4f6c462046fff7ebff72b694e803002b7886e8030043f002033846f5
:020000040800f2
:203860002b70fef7effc62b6ede700bfbc0f0020a40f00201c0500202de9f04fdff8f8807f
:020000040800f2
:203880004468b8f80c30b8f80a60a4eb032486fb046eb8f80630b60946ea8e664fead33cbc
:020000040800f2
:2038a0005b04f618b8f80e20b8f8083082fb04254cebae1c83fb043eb8f80480d20ddb0977
:020000040800f2
:2038c00042ea452243ea4e634fea084813eb080302f5fa674feaee1e4ef1000eb7f5fa6fe6
:020000040800f2
:2038e0004feae55533da84fb0448e40f554344ea4804a2fb02b808eb45083d25abfb059a3a
:020000040800f2
:2039000005fb08aa1beb0b05dff870b04fea191948eb08085f4549ea0a794fea2a1a0ada7f
:020000040800f2
:203920004ff00f0b02f6ac525243c2fb0b9a4ff0080bc2fb0b58b6eb09096ceb0a0a5d1b39
:020000040800f2
:203940006eeb08084e46d4462b46c6463f1b0068a0fb033200fb0e225b0d43eac2239b1be6
:020000040800f2
:203960004fea625262eb0c02db0b43ea4243c1e90037bde8f08f00bfa80f002024faffffb0
:020000040800f2
:2039800037b50d4c694604f11400fff775ff009d61692a46094804f065faa169019a084850
:020000040800f2
:2039a00004f060fa284601f0e9ff0146054803b0bde8304004f056baa80f002030a600085d
:020000040800f2
:2039c00048a6000860a6000810b5114c1148618804f048faa188104804f044fae1880f48d6
:020000040800f2
:2039e00004f040fa21890e4804f03cfa61890d4804f038faa1890c4804f034fae1890b48ad
:020000040800f2
:203a000004f030fa218a0a48bde8104004f02abaa80f00206fa6000884a6000895a6000855
:020000040800f2
:203a2000a5a60008b5a60008c5a60008d6a60008eba6000800230820124a10b51249937472
:020000040800f2
:203a4000124a032b0bd18b6943f004038b611061136823f4704343f4805313600423013358
:020000040800f2
:203a6000202beed10a48fdf723ff0a4a0a490b48fef764fbbde8104041220621084b034869
:020000040800f2
:203a800001f0fabca80f00200010024000080140d0ae0008fba600083b380008c80f00206c
:020000040800f2
:203aa000793600081fb50c490c48b1f90a30b1f902200293b1f9083052425b420193b1f93c
:020000040800f2
:203ac00006300093b1f90430b1f9001004f0caf905b05df804fb00bff011002002a7000834
:020000040800f2
:203ae0004ff0804313b5084c8df804008df8051001222361022101a8fff75cfa4ff48043c0
:020000040800f2
:203b0000236102b010bd00bf001001404ff0005313b5084c8df804008df80510012223611a
:020000040800f2
:203b2000022101a8fff746fa4ff40053236102b010bd00bf0010014073b54ff000531546c5
:020000040800f2
:203b400001220c460a4e60f07f008df80700114633610df10700fff72dfa01222946204638
:020000040800f2
:203b6000fff796fa4ff40053336102b070bd00bf00100140922337b501228df807304ff0e7
:020000040800f2
:203b800080430c4d04462b6111460df10700fff711fa01220df106001146fff779fa0122cc
:020000040800f2
:203ba00006212046fff774fa4ff480432b6103b030bd00bf001001407fb54ff080464ff456
:020000040800f2
:203bc000804507210120fff7a5fab6217e20fff787ff634cb6211420fff798ff0320fef7f2
:020000040800f2
:203be000d3fb00202661fef7cffb01202561fff7a1fa07210120fff78dfa802301228df848
:020000040800f2
:203c0000023011460df102002661fff7d3f90122022103a8fff73cfa25619df80d301e2b14
:020000040800f2
:203c200040f093800122002003a9fff785ff9df80c300f2b40f0898004217d20fff750ff8d
:020000040800f2
:203c40000020fef7a1fb03214120fff749ffac214020fff745ff0020fef796fb0d216d2028
:020000040800f2
:203c6000fff73eff0520fef78ffb01a8fff782ff09216d20fff734ff0520fef785fb03a828
:020000040800f2
:203c8000fff778ff00216d20fff72affbdf90c20bdf904309b1a40f25452934255ddbdf9d4
:020000040800f2
:203ca0000630bdf90e105b1a93424eddbdf91020bdf908309b1a40f2a922934245dd0121e6
:020000040800f2
:203cc0003c20fff723ff0df1030101223c20fff733ff9df803108b07f5d511f0040434d1b5
:020000040800f2
:203ce000a9214020fff7fcfe03214120fff7f8fe21460f20fff70aff06211020fff706ff52
:020000040800f2
:203d00000120fff717fa174c174d07210120fff701fa03a8fff72eff06220df11201022051
:020000040800f2
:203d2000fff70aff0120fff705fa72b603ab03cb206018682b78a06043f004030b486160d9
:020000040800f2
:203d40002b70fef77ffa62b6dfe7094a137843f004031370044a11780b431370d0e700bfc3
:020000040800f2
:203d600000100140f0110020a40f00201c0500205220002038b54ff4804000232049214a44
:020000040800f2
:203d80000e2b0bd18b6943f010038b611061536823f0706343f0807353600f230133202b4c
:020000040800f2
:203da000eed100234ff400501549164a0d2b0bd18b6943f010038b611061536823f47003e0
:020000040800f2
:203dc00043f4801353600e230133202beed14ff080430c4d2b61fef79ffc0446fef79cfca9
:020000040800f2
:203de000031b012bfad94ff4804307482b61074a0749fef7a3f9bde838400648fdf758bd1f
:020000040800f2
:203e000000100240001001400012002023a70008b93b0008f8ae0008054a0648b2f90430d5
:020000040800f2
:203e2000b2f902105b42b2f90020494204f01ab8281400202aa7000813b504460120fff7ae
:020000040800f2
:203e400069fa60210120fff77dfa01220023114601a88df80440fff7adfa61210120fff7ab
:020000040800f2
:203e600071fa012301a81a461946fff705fb0120fff762fa9df8040002b010bd07b58df889
:020000040800f2
:203e8000040001208df80510fff744fa60210120fff758fa012302211a4601a8fff78afa7b
:020000040800f2
:203ea0000120fff749fa03b05df804fb38b5184d04460120fff72efa60210120fff742faf2
:020000040800f2
:203ec000002301222846114600f8063ffff772fa61210120fff736fa012306211a46e81dbf
:020000040800f2
:203ee000fff7cafa0120fff727fab5f807305bbaa3f500432380b5f809305bbaa3f5004383
:020000040800f2
:203f00006380b5f80b305bbaa3f50043a38038bd2814002010b5012104460920fff7aeff75
:020000040800f2
:203f20000820fff789ff10f0010002d1fef72cfaf6e72046bde81040b8e700234b4c83b523
:020000040800f2
:203f400080210a206373fff799ff0120fef71cfa2f20fff771ff3038c0b20128444d07d9dd
:020000040800f2
:203f6000444a137843f0080313702a7813432b700a20fef709fa08210920fff77fff0a20c2
:020000040800f2
:203f8000fef702fa3c48fff7c5ff0a20fef7fcf910210920fff772ff0a20fef7f5f9374891
:020000040800f2
:203fa000fff7b8ffb4f91420b4f90e300121134403ebd3735b10b4f916206383b4f91030ba
:020000040800f2
:203fc0000a20134403ebd3735b10b4f91820a383b4f912302a4f134403ebd3735b10e383f2
:020000040800f2
:203fe000fff74cff0e210b20fff748ff0123254e6373637b13b16846fff758ffbdf90030f9
:020000040800f2
:20400000b4f91a20b4f91c109b1a47f6ff729342a8bf1346bb42b8bf3b46adf80030bdf968
:020000040800f2
:2040200002305b1a9342a8bf1346bb42b8bf3b46b4f91e10adf80230bdf904305b1a934269
:020000040800f2
:20404000a8bf1346bb42b8bf3b46adf8043072b6bdf804300098a3802b78206043f00803a5
:020000040800f2
:2040600030462b70fef7eef862b6c2e728140020a40f002052200020361400203c140020f8
:020000040800f2
:204080000080ffff1c05002008b500230548064a437306492030fef751f8bde80840044818
:020000040800f2
:2040a000fdf706bc281400203da700083b3f000820af00081fb54ff4667340f20162cde96e
:020000040800f2
:2040c0000132074907488b680093b1f90430b1f90220b1f9001003f0c5fe05b05df804fb65
:020000040800f2
:2040e0007016002045a7000808b503213420fff711f84ff08052014b1a6108bd0010014004
:020000040800f2
:2041000007b58df804008df80510fff7edff022101a83422fef74eff4ff48052034b3420c3
:020000040800f2
:204120001a61fff707f803b05df804fb00100140f22313b504468df80030fff7d5ff694662
:020000040800f2
:20414000342308460722fef7bdff4ff48052064b34201a61fef7eeffddf801302360bdf88b
:020000040800f2
:204160000530a38002b010bd0010014073b5002504460e46c0e9005585606846fff7d8ffce
:020000040800f2
:20418000bdf900202368012013442360bdf902206368013513446360bdf90420a368134494
:020000040800f2
:2041a000a360fef7f1f8ae42e7d102b070bdf0b50b2187b03120fff7a3ff80238df80c3042
:020000040800f2
:2041c000fff792ff03a9084634230222fef77aff4ff48052354b34201a61fef7abff9df8dd
:020000040800f2
:2041e0000d30334ce52b07d0324a137843f0100313702278134323700b212c20fff780ffdc
:020000040800f2
:2042000000211e20fff77cff00211f20fff778ff00212020fff774ff00212e20fff770ff63
:020000040800f2
:2042200000213820fff76cff08212d20fff768ff04216846fff79aff0a216846fff796ff0b
:020000040800f2
:204240008b213120fff75cff042103a8fff78eff0a2103a8fff78aff0b213120fff750ffa6
:020000040800f2
:20426000029a059b9b1a144ab3f5667f936007da104a137843f0100313702278134323705d
:020000040800f2
:204280000421eff310856846fff770ff0a4f0b4e3846fff74dff72b62378304643f010037e
:020000040800f2
:2042a0002370fdf7cfff85f31088f1e700100140a40f002052200020701600201c05002024
:020000040800f2
:2042c00008b51048fdf7f4fa00234ff480500e490e4a0c2b0bd18b6943f010038b61106158
:020000040800f2
:2042e000536823f4702343f4803353600d230133202beed1064a07490748bde80840fdf77e
:020000040800f2
:204300001dbf00bf48af000800100240001001407ba70008af41000880160020f8b51d4d71
:020000040800f2
:204320001d4c2b78002043f001032b70fef7a8fc22782b78d2b21f2b28d1184e184906eb2a
:020000040800f2
:20434000821303f1180503c985e80300154934330868898843f80c0c23f8081c12499701b0
:020000040800f2
:204360000d68898843f8065c104d23f8021c28686968013203c3a86802f01f0218600c4b38
:020000040800f2
:2043800020461b68f3512270fdf786ff0122094b1a70f8bda40f0020a0070020a4070020ca
:020000040800f2
:2043a000bc0f00202814002070160020f011002018050020a818002000b599b008a8fff72e
:020000040800f2
:2043c0002df9bdf93430bdf924200693bdf9323008990593bdf930300a480493bdf92e30a6
:020000040800f2
:2043e0000393bdf92c300293bdf92a300193bdf928300093bdf9263003f034fd19b05df8ed
:020000040800f2
:2044000004fb00bf83a7000837b5124b1a78f2b1114d002429461c70104b41f84c4b1878f6
:020000040800f2
:204420004ff416530e4a009302eb801209232046fef7ccfb20460b49fef70afc2046fef708
:020000040800f2
:204440000dfc094bab60ab6003f58003ab6003b030bd00bfa818002000240140a0070020f8
:020000040800f2
:20446000a80700201d43000801018e0008b5434b00209a6942f010029a61414a116821f4af
:020000040800f2
:2044800070211160996941f010019961116821f470011160996941f010019961116821f4a0
:020000040800f2
:2044a00070411160996941f010019961116821f470611160996941f010019961116821f004
:020000040800f2
:2044c000f0011160996941f010019961116821f00f0111609a6942f008029a61294a11680b
:020000040800f2
:2044e00021f00f011160996941f008019961116821f0f00111609a6942f400729a614ff41f
:020000040800f2
:204500008072214b98605a60204ada606ff040421a614ff40002da625a6b42f00e025a6346
:020000040800f2
:204520005a6b42f4f0725a635a6b42f450525a635a6b42f4c0225a635a6b42f430025a6383
:020000040800f2
:204540005a6b42f0a0525a631a6b42f008021a631a6b42f490721a631a6b42f480421a6343
:020000040800f2
:204560009a6842f400029a601860fef7bbfb0848fdf79ef90122074b1a7008bd00100240f3
:020000040800f2
:2045800000100140000c014000240140ffff030070af0008a8180020164a174968b94ff0f0
:020000040800f2
:2045a00080431860d36923f00103d3610b6823f4706343f400730b6070470b6823f47063b3
:020000040800f2
:2045c00043f420630b60d369602143f00103d3614ff0804300225a6099629a603022d8622f
:020000040800f2
:2045e000d863da614ff480721a6201221a605a61704700bf001002400008014010b50c4614
:020000040800f2
:20460000fff7caff2046fdf7bffebde810400020fff7c2bf0c4a0d49536823f44073536054
:020000040800f2
:204620000b4a936943f0040393614ff480230b610b6823f4706343f480730b60d36923f068
:020000040800f2
:204640000103d361704700bf00000140000801400010024008b500f088fa074b074819687f
:020000040800f2
:2046600003f000fc064b0748196803f0fbfbbde8084000f089ba00bf38190020e0a7000862
:020000040800f2
:204680003c190020f3a700082de9f04106460f46154600f06afa124b1b68b34202d800209d
:020000040800f2
:2046a000bde8f081aa199342f9d3dff838800db90120f5e7b8f800403946631e3340e41acd
:020000040800f2
:2046c000a4b2ac4228bf2c463046224600f00efa0028e4d02d1b2744adb22644e7e700bf82
:020000040800f2
:2046e00038190020441900202de9f84ffdf770f81d4b04461f78afbb1c48fef790f84ff040
:020000040800f2
:204700000208dff86ca02402802251463819fff7bbffd0b10025dff858b0781980b2fcf711
:020000040800f2
:20472000b7ff08260beb05092020fdf74bff013e19f8010bfcf7a2ff16f0ff06f4d10a2029
:020000040800f2
:204740000835fdf73fff802de7d1b8f1010f4ff0800704d1bde8f84f0448fef77db84ff090
:020000040800f2
:204760000108d1e7bde8f88fec000020a9180020aa1800202de9f04106460f46154600f04a
:020000040800f2
:20478000f4f9124b1b68b34202d80020bde8f081aa199342f9d3dff838800db90120f5e791
:020000040800f2
:2047a000b8f800403946631e3340e41aa4b2ac4228bf2c463046224600f058f90028e4d000
:020000040800f2
:2047c0002d1b2744adb22644e7e700bf38190020441900202de9f041054600f0c6f9144845
:020000040800f2
:2047e000fef71df8134bdff850801e6836b901240f48fef731f82046bde8f081802e3746f4
:020000040800f2
:2048000028bf802741462846bab2fff73dff04460028edd00023084a12f8011bff2905d1af
:020000040800f2
:2048200001339f42f8d13d44f61bdfe70024dfe7a91800203c190020aa180020f8b50e4f16
:020000040800f2
:204840003b685c1e0c44b4fbf3f45c43c01a05190cb901200be004262846fff7bbff38b9b4
:020000040800f2
:20486000284600f0cbf810b1013ef5d13046f8bd3b68ed1ae41aebe73c19002008b5fcf787
:020000040800f2
:204880001fff0648fcf7e4ff30b1054b00201968bde80840fff7d2bf08bd00bfd6a5000889
:020000040800f2
:2048a0004019002008b5fcf793ff054b1b7833b9044b00021968bde80840fff7bfbf08bd76
:020000040800f2
:2048c000ec0000203c19002008b500f073f9bde808400148fcf7ecbfa0af0008012170b5cc
:020000040800f2
:2048e00004460b4e0846fef715fc0122230433610623084d114628462b70fef75bfb346125
:020000040800f2
:204900000120fef717fcab881c43ac8070bd00bf000c01402c19002038b5174c0546a3884c
:020000040800f2
:20492000da0421d501210846fef7f4fb4ff08052124b20461a610122052311462370fef7d6
:020000040800f2
:2049400039fb012220461146fef7a2fb2378db07f7d44ff48052094b01201a61fef7eafb8a
:020000040800f2
:20496000a38823f48053a3802b0c63702b0aa370e5704ff4805038bd2c190020000c01409e
:020000040800f2
:2049800038b51c4ca368f3b901210846fef7c2fb4ff08053184d01222b619f231146204644
:020000040800f2
:2049a0002370fef707fb012204212046fef770fb4ff4805301202b61fef7bcfb2378ff2b2b
:020000040800f2
:2049c00002d10023a36038bda378a3f111020e2af7d8a3f1100201239340a3601b04e3601e
:020000040800f2
:2049e000a3f580334ff4803263614ff4807322612383e8e72c190020000c014070b5194c49
:020000040800f2
:204a00000546e26882422ad9236903449a4226d304f11a00fdf703fffff7b2ff2846fff782
:020000040800f2
:204a20007bff0546fff75aff0121d82308460e4e2370fef76ffb2b04012204213361204638
:020000040800f2
:204a4000fef7b8fa01203561fef774fba38804f11a001d43a580fdf7fffe012070bd002076
:020000040800f2
:204a6000fce700bf2c190020000c01402de9f0411c4c0546e3680f46834216462fd90244d9
:020000040800f2
:204a800093422cd304f11a00fdf7c9fefff778ff2846fff741ff0546fff720ff01210223c0
:020000040800f2
:204aa0000846dff844802370fef734fb2b04c8f81030012204212046fef77cfa0122314674
:020000040800f2
:204ac0003846fef777fa0120c8f81050fef732fb04f11a00fdf7c0fe0120bde8f081002077
:020000040800f2
:204ae000fbe700bf2c190020000c01402de9f0411b4c0546e3680f46834216462dd902445d
:020000040800f2
:204b000093422ad304f11a00fdf789fefff738ff2846fff701ff0121054603230846dff8f0
:020000040800f2
:204b200044802370fef7f6fa2b04c8f81030012204212046fef73efa012231463846fef722
:020000040800f2
:204b4000a7fa0120c8f81050fef7f4fa04f11a00fdf782fe0120bde8f0810020fbe700bf15
:020000040800f2
:204b60002c190020000c0140704710b5054c2046fdf755fefff704ff2046bde81040fdf7c1
:020000040800f2
:204b80006bbe00bf4619002038b5084c04f11a052846fdf744fefff7f3fe2846fdf75cfe12
:020000040800f2
:204ba000a1680348bde8384003f05cb92c1900200ca8000800234ff480500a490a4a0c2b47
:020000040800f2
:204bc0000bd18b6943f008038b611061536823f4702343f4803353600d230133202beed1fa
:020000040800f2
:204be000704700bf00100240000c014070b572b60c4e049d56f8204041ea422104f4804262
:020000040800f2
:204c000084ea0515114304f0400284ea0334114304f4405405f030052143294346f8201095
:020000040800f2
:204c200062b670bd005c0040044b1a78012a9fbf511c19709b185870704700bf48190020c1
:020000040800f2
:204c400030b50024a3b2d51aadb2012d10d85308c3ebc33402eb440292b242b110f81320ed
:020000040800f2
:204c600051f8230000f47f40024341f8232030bd055b5b0841f823500234e3e7002370b5b0
:020000040800f2
:204c8000461c9cb2151badb2012d0bd85308c3ebc33402eb440292b21ab151f8232000f8fe
:020000040800f2
:204ca000132070bd640851f82440c454c4f30724f4540233e5e770b5144ce378f3b100268e
:020000040800f2
:204cc000134d04f11000237962799a4219d1a379a3b1a368a671da6ad2b2627112b1e168f9
:020000040800f2
:204ce000fff7ccff2671ab6823f40f639b049b0c83f4304383f08003ab60e4e74ff0ff3056
:020000040800f2
:204d000070bd5a1c22711c44207cf9e748190020005c004038b5114dab68686ddc6895f860
:020000040800f2
:204d20005030c4f309049c4228bf1c461b1b85f850301cb12246a96dfff7a0ff20446865c4
:020000040800f2
:204d400072b6074a136823f40f639b049b0c83f4304383f08003136062b638bd48190020af
:020000040800f2
:204d6000005c004038b5154c04f15c0594f85c30fbb9012394f85d50216e402d84f85c30c6
:020000040800f2
:204d800002d084f864301db12a460d48fff758ffa3680c4a5d63002384f85d30d36823f0b6
:020000040800f2
:204da000c0035b055b0d83f4004383f0b003d36038bd2846fdf746fad8e700bf48190020bf
:020000040800f2
:204dc000ad190020005c004010b5064ce37823b172b694f864300bb162b610bdfff7c2ff6b
:020000040800f2
:204de000f7e700bf4819002070b5114c0546e378abb172b604f15c0694f85d203f2a12d836
:020000040800f2
:204e0000002384f86430531cdbb284f85d30402b144484f8655001d1fff7a4ff62b670bdb6
:020000040800f2
:204e20003046fdf70ffa94f85c30002bf8d1e3e748190020174b70b51b6803f03003302b1d
:020000040800f2
:204e400027d0154c2378d4f8a8601f2b96bf1d4620250022a3eb050398bf84f8a520237061
:020000040800f2
:204e60002db12a463046d4f8ac10fff7e9fea3682e44c4f8a8605d6072b6064a136823f005
:020000040800f2
:204e8000c0035b055b0d83f4004383f0b003136062b670bd005c0040481900202de9f74f76
:020000040800f2
:204ea0000025b34c10f00107064684f8b05039d04022b04b29461d65af4b2846a3601a60c2
:020000040800f2
:204ec00003f180025d60c4f8ac2060229a604ff40042c03343f8b42ca3658023a4f8b230df
:020000040800f2
:204ee0000223012200930323fff780fe00233846012219460095fff779fe0130c7b2082f37
:020000040800f2
:204f0000f4d180229b4bda6484f8b450e57084f8a550c4f8a8502570656584f8505003b0de
:020000040800f2
:204f2000bde8f08f810730d504f1b6036365082384f85030fff7eefe94f850302bbb94f9c2
:020000040800f2
:204f4000b62094f8b630002a48dbb4f8bc20002a0cbf0122022284f8a520884a13f0600082
:020000040800f2
:204f6000c4f8a8204ff00002227039d0202800f0eb8094f8a530012b07d1b4f8bc30227897
:020000040800f2
:204f80009a4288bf2370fff755ff720710d594f8a530022b0cd1fff7bdfe94f850303bb997
:020000040800f2
:204fa000012284f8a520227802b12370fff742ff3307b4d594f8b43043b194f8be306d4a1e
:020000040800f2
:204fc00043f08003d364002384f8b43094f8a530012ba4d103b0bde8f04f2be70122bae7f2
:020000040800f2
:204fe00003f01f03012b00f09d80022b00f0a180002bbed194f8b730092bbad801a252f845
:020000040800f2
:2050000023f000bf3d510008734f0008734f0008734f0008734f00082d5000083d500008e6
:020000040800f2
:20502000734f0008795000087f500008b4f8b83084f8be30012384f8b4309ae7b4f8b83067
:020000040800f2
:205040004f491d0a2f46dbb20a78002a91d04878b8420fd1581ec0b25bb9022d08bf8a78f4
:020000040800f2
:20506000b4f8bc30c4f8a810934238bfdab222707fe703461144e7e794f8bf0061e00025b7
:020000040800f2
:205080004ff0020b0121d4f80880b4f8b270b4f8b830c8f8107084f8bf3008462b46c8f8c2
:020000040800f2
:2050a00014500322cdf800b0fff7a0fd4ff40443dff8c4a007f108091ffa89f9c8f828907e
:020000040800f2
:2050c000c8f82c300aeb490307f14809e3602a4658461ffa89f9032304210095fff786fde5
:020000040800f2
:2050e00088370aeb4903c8f8309023662a462b460521c8f83450a4f8b2700320cdf800b006
:020000040800f2
:20510000fff774fd1f4884f8645084f85c50fdf7c3f801231c48a57184f8bf50e370fdf74a
:020000040800f2
:20512000bbf826e794f8b73043b10a2b7ff421af07e094f8b730002b7ff41baf0020fff7f8
:020000040800f2
:2051400073fdfff771fd14e794f8b730202b08d0212b7ff40eaf0d4bc4f8a83007232370c5
:020000040800f2
:2051600007e70a4b6365072384f8503001e700bf48190020005c0040006000404919002018
:020000040800f2
:2051800036110008a41900204b190020200000203c494b6c180460d540f20f7003f00f03dc
:020000040800f2
:2051a00051f82320104041f82300032b68d8dfe803f0023a1f2d344bb3f8c0100131a3f840
:020000040800f2
:2051c000c010110409d593f8b01010054cbf41f0020141f0040183f8b010120642bf93f858
:020000040800f2
:2051e000b02042f0080283f8b02093f8b00055e6254b1004b3f8c21001f10101a3f8c21080
:020000040800f2
:205200003ed5012221489a71fdf746b81e481106b0f8c43003f10103a0f8c43030d500232d
:020000040800f2
:2052200000f85c3ff0e718491206b1f8c63003f10103a1f8c63023d512494a6882f02003cb
:020000040800f2
:2052400022f0f002520503f03003520d134343f4004343f080034b6070475b0510d50a4bec
:020000040800f2
:20526000b3f8c8200132a3f8c8204a6c22f480624a6493f8b00040f0010083f8b000b6e755
:020000040800f2
:20528000704700bf005c00404819002014050020024a536c23f4805353647047005c004043
:020000040800f2
:2052a00010b572b6054cfff706fd431c02d062b6c0b210bd2046fcf7c5fff4e714050020fe
:020000040800f2
:2052c00072b60122094b4ff080711a6400225a6402f1804202f58432116103221a64044adc
:020000040800f2
:2052e000d36923f40003d36162b67047005c0040001002404ff080731449154a0b61d369d1
:020000040800f2
:2053000043f40003d36172b6124a0120d2f8143323f0ff0343f0c003c2f814334ff4801387
:020000040800f2
:20532000136000220c4b83f8bf200c4b18641a645a644ff404421a6462b64ff47a7300bf0a
:020000040800f2
:20534000013bfcd14ff480730b617047000801400010024000e100e048190020005c004072
:020000040800f2
:20536000104a10b5936949f6404443f0040393614ff080730c4a1361536823f00f0343f012
:020000040800f2
:205380000103536000bf013cfcd1fff7b3ff074b074a83f8a54007490748bde81040fdf75a
:020000040800f2
:2053a0004db900bf001002400008014048190020c94d0008e94d0008b74c00080123084930
:020000040800f2
:2053c00010b44c69074a8340234014604b612bb102eb800253680bb110bc184710bc70474d
:020000040800f2
:2053e00000040140141a0020174b2de9f0475e69164d04462e601640b5f844200f46b242b9
:020000040800f2
:2054000008d15a6195f8463005eb83035b68bde8f04718474ff001095e6105f10408e3b2e2
:020000040800f2
:205420009f4201d2bde8f08726fa04f2d20709d558f8242032b109fa04f1a5f8441085f8f2
:020000040800f2
:20544000463090470134eae700040140141a00200020b3e70120b1e70220afe70320ade784
:020000040800f2
:205460000420abe74ff4787209210520bce74ff47c420f210a20b7e72de9f0410127684c3b
:020000040800f2
:20548000dff8a0e104eb81048d007045636007fa01f64feaa10405f00c0800f08e80624bb1
:020000040800f2
:2054a000984200f08c8003f58063984200f0898003f58063984200f0868003f58063a0eb57
:020000040800f2
:2054c000030cdcf1000343eb0c039b004ff00f0ca40004f1804404f58034a7680cfa08fc98
:020000040800f2
:2054e00027ea0c0703fa08f33b435706a3602dd470456ad14d4ca36943f00403a361002ab4
:020000040800f2
:2055000000f08480042a14bf0123002301f1100403fa04f30cbf012400248c4023430361ab
:020000040800f2
:20552000022305f01c04032504f102084fead10c50f82c7005fa08fea5404eea050427ead4
:020000040800f2
:20554000040403fa08f3234340f82c30f043384bd5071c6824ea06041c609c6854bf04404c
:020000040800f2
:2055600034439c6094074bbfd868dc68304320400429d8604cd80631c9b2d0064dd412f088
:020000040800f2
:20558000200f14bf40238023ff262a4c8a10c032c80054f8225000f01800864025ea06056e
:020000040800f2
:2055a00083402b4344f8223001234a1101f01f018b4044f82230bde8f081002386e73b461c
:020000040800f2
:2055c00084e7022382e7032380e7174b984204d1164ca36943f0080390e7174b984204d100
:020000040800f2
:2055e000124ca36943f0100388e7144b984204d10e4ca36943f0200380e7114b98427ff4b2
:020000040800f2
:205600007eaf0a4ca36943f0400377e7012388e709298cbf28211721afe7c023b4e700bfc3
:020000040800f2
:20562000141a002000080140000c0140001002400004014000e100e0001001400014014088
:020000040800f2
:2056400000180140012303fa01f1084b12f0010f986814bf08438843986012f0020fda6843
:020000040800f2
:2056600014bf0a438a43da60704700bf00040140024b03eb81035a60704700bf141a00200b
:020000040800f2
:20568000012303fa01f1034b59611a680a431a60704700bf00040140012303fa01f1034b8a
:020000040800f2
:2056a0001a6822ea01021a605961704700040140704700bf38b504460e4d95f8f80074b177
:020000040800f2
:2056c000013ce4b2142195f8f800013cfef796ffe4b21420fcf758feff2cf3d105e032213c
:020000040800f2
:2056e000fef78cff1420fcf74ffebde838401e20fcf74abe1803002030b50a21002485b0bc
:020000040800f2
:2057000020eae070234603f110020deb020590fbf1f201fb1200013405f80c0ce4b210460f
:020000040800f2
:20572000002aefd101aad518013ce4b215f80109fff7c0ff002cf7d105b030bd10b50020cd
:020000040800f2
:20574000fdf75ef904460120fdf75af9431e584204f1ff3258415442544144ea400010bd2c
:020000040800f2
:20576000f8b5fff7ebff3d4d00285ad04b275e260138c4b295f8f80002217843b0fbf6f027
:020000040800f2
:20578000013cc0b2fef73affe4b20a20fcf7fcfdff2cefd11920fcf7f7fd002496265e2710
:020000040800f2
:2057a000e0b201f03bfc012817bf95f8f80095f8f8007043b0fbf7f00ebf0221c0b202215c
:020000040800f2
:2057c000fef71cff01341420fcf7defd042ce7d100f0e1fa20b30a20fcf7d6fd0226962727
:020000040800f2
:2057e0005e2495f8f8000a217843b0fbf4f0c0b2fef704ff0a2195f8f800fef7fffe4b23b3
:020000040800f2
:2058000095f8f8000a215843b0fbf4f0c0b2fef7f5fe0a2195f8f800fef7f0fe012e1bd1a6
:020000040800f2
:20582000f8bd05244b275e2695f8f80002217843b0fbf6f0c0b2fef7e1fe962395f8f8001c
:020000040800f2
:2058400002215843b0fbf6f0013cc0b2fef7d6fe14f0ff04e8d19de70126c2e71803002032
:020000040800f2
:205860002de9f041384d394e90b02b78337083bb374c6846fdf7d2febdf9100018b920461f
:020000040800f2
:20588000fcf7e0fcf5e700f095f8fff735ff3378092b04d12f4b187808b1fff72dff337872
:020000040800f2
:2058a000082b33d12c4b1c682c4b93f8fc3043b127235c430c2394fbf3f414b10020fff72b
:020000040800f2
:2058c000f9fe2046fff718ff4ff4fa70fcf75cfdcbe7234ad75c002fd9d0dff8808007f06d
:020000040800f2
:2058e0000704013ce4b2ff2c03d12420fcf74cfdcde73b074cbf1421062198f8f800fef771
:020000040800f2
:205900007dfe0620fcf740fd7f08eae7012b01d1fff726ff2b78022b07d032782b789a4275
:020000040800f2
:20592000a3d12846fcf78efcf7e7fff719ff32242b78022beed10a20013cfcf725fd14f0b7
:020000040800f2
:20594000ff04f5d1e6e700bf50200020601a0020ec1f002052200020382000201803002058
:020000040800f2
:205960002eb00008024a03490348fcf7e7bb00bf27a8000861580008681a00200b4b0c4a24
:020000040800f2
:205980009842a8bf184620eae070031210b552f82340013352f82330c0b2c0f58071584303
:020000040800f2
:2059a00004fb01008030001210bd00bfc0d4010038b0000841f21c435843044b00f547302c
:020000040800f2
:2059c00000f2ce3090fbf3f000b270479c3f0600034a044b92691b6850435b4218407047c6
:020000040800f2
:2059e000180300203c190020044b00f580701b680422034903eb8000fef746be40190020ee
:020000040800f2
:205a0000901c0020fff7b0b808b55523084900f580700b708b8804224b80064b1b6803ebb0
:020000040800f2
:205a20008000fef7a7febde80840fff79db800bf901c00204019002020235a20074a12f8f8
:020000040800f2
:205a4000011b013b084413f0ff03c0b2f7d14042c0b2b0fa80f04009704700bf981c0020c2
:020000040800f2
:205a600038b50446fff7b4fffef7b4fea0b90b4b0b4d98692022604305f10801fef704febc
:020000040800f2
:205a800008b9e04338bdfff7d7ff0028f9d02b7a462bf6d1a889f5e70020f3e71803002051
:020000040800f2
:205aa000901c002070b500260b4b35461c680b4b9b69b4fbf3f4e4b2f0b2844201d8284645
:020000040800f2
:205ac00070bdfff7cdff002803dd0db1854200da85b20136f0e700bf4019002018030020b8
:020000040800f2
:205ae0002de9f041fbf7ecfd2b4b1b782d2b15d1fbf78cfd4ff0ff34fbf784fe274b1d78d5
:020000040800f2
:205b0000002d47d1264b44431e68264b9b6913d12146bde8f041244802f0a4b90124ebe77a
:020000040800f2
:205b20004046fff771ff21e00134802c12d1fcf741f81be01d4827e0b6fbf3f6f6b2b542e8
:020000040800f2
:205b4000e6d02846fff78cff6f1ca042ffb21fd10024174e5ffa84f84046fff745ff3378c9
:020000040800f2
:205b6000552bddd17288b3889a42ddd12846fff72fff04463846fff72bff011b2046fef747
:020000040800f2
:205b80005dfe0028d6d00b48bde8f04102f082b93d46d4e7bde8f081eb000020ec0000201b
:020000040800f2
:205ba00040190020180300202ea800084aa80008901c002043a800082de9f843194b1a4f7c
:020000040800f2
:205bc0001e68bb690025b6fbf3f6dff86080dff86090f6b2ecb2a64204d8bde8f843154897
:020000040800f2
:205be00002f058b92046fff73bff01460134e0b261b1fff7edfec0f30f234846ba696a43c8
:020000040800f2
:205c0000c2f30f2202f02ef90135e3e7fff7e0feba69c0f30f236a4329464046c2f30f2221
:020000040800f2
:205c2000f0e700bf401900201803002076a800085aa8000890a800082de9f041fcf7e8f98f
:020000040800f2
:205c4000fff730ff294ca080fef78fffa38823b101339bb2002b3fd0a3808025013dedb2a8
:020000040800f2
:205c6000ff2d0dd02846fff7bffe2378552bf5d1a38862881bb1d31a1bb2002b04dda28050
:020000040800f2
:205c8000a3880bb90123a3800023dff86480c4e90a33184ba5881e68d8f81830013db6fbe9
:020000040800f2
:205ca000f3f6f6b295fbf6f306fb1355edb22f463846fff7d5fe7b1cdbb278b9d8f81820b9
:020000040800f2
:205cc00018467a43e262fff783fea0620a48fcf7e3fa0020bde8f0810123bde79e428cbfa1
:020000040800f2
:205ce0001f460027af42e3d1f0e700bf901c00201803002040190020941c0020012302481f
:020000040800f2
:205d000000f8303ffcf7c8ba901c00200022024b83f83020fef728bf901c002038b50023e9
:020000040800f2
:205d20000546437002465a2300f1200112f8010b03449142dbb2f9d1114c5b426b7004f13d
:020000040800f2
:205d40003100fcf76cfdd4e90a329a420ad394f830302bb900240b48fcf77efd204638bdf4
:020000040800f2
:205d6000fff7d4ff94f83030002bf3d0e06a20222946fef7fffce36a2033e3620124eae7ba
:020000040800f2
:205d8000901c0020c11c002008b5fff78bfe003818bf012008bd034bd86a9b6ac31a5842fd
:020000040800f2
:205da00058417047901c0020002310b5084c094884f83030092384f83230fbf779fd04f1f7
:020000040800f2
:205dc0003800054a0549bde81040fcf7b7b900bf901c002090b7000895a80008e15d000831
:020000040800f2
:205de0002de9f74ffef7c1fefff726ffdff8909199f80030002b5dd04623624cdff8888170
:020000040800f2
:205e00002370624b20461b68614e6380614b624d1b88e380614b1b88a381614b1b88e38140
:020000040800f2
:205e2000604b1b882382604b1b6863615f4b1b68a3615f4b1b68e3615e4b1b68a3605e4b03
:020000040800f2
:205e40001b88a380fff76aff5c4b1b78013303f01f0388f800309b01f7580023ba462b7041
:020000040800f2
:205e6000564a98f800301278934227d1544b2a781b789a4211d02b7053232370fcf74cfcfb
:020000040800f2
:205e80002b786080a38000232046e380fff746ff2b78082b01d1fff739fffff7b3fd0a208f
:020000040800f2
:205ea000fcf772fa99f80030002bd9d13448fcf7c9f9f7e74846fcf7c5f999e7990156f837
:020000040800f2
:205ec00001b006eb8310abeb070cbcf1000fa4f802b02cdb412727708769cde90031676036
:020000040800f2
:205ee000c769a760878ea781c78e7f42e781078f2782478f6782878f7f42a782c78fe782f3
:020000040800f2
:205f0000478d7f422783078d6783878d7f42a783fdf79cfbe0832046fff700ffdde9003185
:020000040800f2
:205f20002878052894bf0bf101070bf10a07abeb0a0000281cdb542031442070088a498a93
:020000040800f2
:205f4000204ae180062121810021a0805b01581806eb400080880131062922f8020ff6d114
:020000040800f2
:205f6000194b20461b880bf1200ae383fff7d6fe98f80030013303f01f0388f800306fe74f
:020000040800f2
:205f8000c01c0020981c0020f41e0020f01f0020a4070020cc1f0020c21c0020d81f0020e5
:020000040800f2
:205fa000da1f0020dc1f0020e81f0020e01f0020e41f0020d01f0020941c0020a00700209e
:020000040800f2
:205fc00050200020a01c002004250020154b1968b3f904200a441a60d3e902210a449a606c
:020000040800f2
:205fe0001969b3f914200a441a619969b3f91c200a449a61196ab3f924200a441a62996a03
:020000040800f2
:20600000b3f92c200a449a62196bb3f934200a441a63996bb3f93c200a449a63da8f0132fc
:020000040800f2
:20602000da877047f81e00200022074bb3f9400003f142010132402a21f8020bfad10022cb
:020000040800f2
:2060400083f8c220704700bff81e00202de9f041184cd4f8d010d4f8cc80084601f02efb60
:020000040800f2
:2060600041460546404601f029fb0146284601f01bfad4f8c87005463946384601f01efba2
:020000040800f2
:206080000146284601f010fad4f8c46005463146304601f013fb0146284601f007fa03f08f
:020000040800f2
:2060a00035f9054901f00afb01f0cefca4f84000bde8f081f81e0020e12e654238b514468e
:020000040800f2
:2060c0000d4603f081fa0146286001f0f7fa01464ff07e5001f0e8f903f0c8f8206038bd00
:020000040800f2
:2060e0002de9f047d1f80090d1f804808f68ce6804460d464846494601f0e0fa41468246ac
:020000040800f2
:20610000404601f0dbfa0146504601f0cff939468246384601f0d2fa0146504601f0c6f98e
:020000040800f2
:2061200031468246304601f0c9fa0146504601f0bdf90021824601f07dfce8b1504603f0fd
:020000040800f2
:2061400095f801464ff07e5001f06cfb4946054601f0b4fa41462060284601f0affa3946ff
:020000040800f2
:206160006060284601f0aafa3146a060284601f0a5fae060bde8f08795e80f0084e80f0084
:020000040800f2
:20618000f8e72de9f04f0025724c87b02368a0685b124012a4f8d4302560c4f8d800fff7b0
:020000040800f2
:2061a000edfb2369a5605b12a4f8e030a36925615b12a4f8e230236aa5615b12a4f8e430f0
:020000040800f2
:2061c000a36a2562c4f8e830236ba562c4f8ec302563a36ba563604dc4f8dc00c4f8f0302b
:020000040800f2
:2061e000fff722ffb5f9f430b4f9e200c01a01f011fab5f9f6300746b4f9e400c01a01f0d4
:020000040800f2
:2062000009fab5f9f2300646b4f9e000c01a01f001fa002302a90590084602930397049692
:020000040800f2
:20622000fff75eff6b7f002b00f09080dff82c81059b00211846019301f040faddf810901f
:020000040800f2
:2062400005464946404601f039fa0146284601f02bf9ddf80ca007465146404601f02efaec
:020000040800f2
:20626000294601f021f900210646484601f026fa00218146504601f021fa82460146484671
:020000040800f2
:2062800001f012f939460546384601f017fa31468346304601f012fa0146584601f006f930
:020000040800f2
:2062a00029468346284601f009fa0146584601f0fdf802f0dbff51468346484601f0f6f8e0
:020000040800f2
:2062c000019b81461946404601f0f8f90146484601f0ecf84ff07e51804601f0e7f84ff007
:020000040800f2
:2062e0007c5101f0ebf902f0c1ff414681464ff07e5001f0d9f84ff07c5101f0dff902f066
:020000040800f2
:20630000b5ff594601f08efa80460146384601f0d5f94146c4f8c800304601f0cff94146a6
:020000040800f2
:20632000c4f8cc00284601f0c9f90d49c4f8d0000846c4f8c490fff7d3fefff787fefff73c
:020000040800f2
:2063400073fe0023e38707b0bde8f08f4ff07e586ee700bff81e002018030020000080bf8b
:020000040800f2
:20636000bc1f00202de9f04f314889b0fbf794ff3048fbf767ff304f2e4a97f8f440127882
:020000040800f2
:20638000944207d197f80401b0fa80f0400909b0bde8f08f2948a201815800eb8414c7f84c
:020000040800f2
:2063a000f81002f12001183201441044fdf764fa206af860fff7e2fad7f8dc20c7f8fc0052
:020000040800f2
:2063c000801ac7f800012046fdf740f9a28eb880ba82e28e5242ba83228fba84a28f524237
:020000040800f2
:2063e000ba85e28fba86628fba8797f804215ab3fa8fb2f5007f09d2fff7e8fd97f8f420b2
:020000040800f2
:20640000013202f01f0287f8f420b4e70c494a8a8988521a0b4912b2a7f8062191fbf2f214
:020000040800f2
:20642000c7f80821fff7adfe002287f80421e5e7ec1f0020a0070020f81e0020a40700204e
:020000040800f2
:206440001803002014d03901a84a1278022a06d8fa8fb2f5007f80f04081fff7b7fd00f0e3
:020000040800f2
:20646000a7f9d7f8ec20b7f93400c2eb402001f0d1f84ff06c5101f021f99d4901f01ef901
:020000040800f2
:206480009c4901f01bf9d7f8f0200546b7f93c00c2eb402001f0bef84ff06c5101f00ef954
:020000040800f2
:2064a000934901f00bf9934901f008f90446d7f8e820b7f92c00c2eb402001f0abf84ff060
:020000040800f2
:2064c0006c5101f0fbf88a4901f0f8f8894901f0f5f803aa02a9fff7f1fd284605aa04a9b1
:020000040800f2
:2064e000fff7ecfd07aa204606a9fff7e7fd039eddf814b03046594601f0e0f8029dddf891
:020000040800f2
:2065000010a080465146284601f0d8f8079c00902146404601f0d2f8ddf8189001904946c7
:020000040800f2
:20652000009801f0cbf80146019800f0bfff29460190584601f0c2f851460546304601f0ef
:020000040800f2
:20654000bdf829468246204601f0b8f851460646484601f0b3f80146304600f0a5ff514653
:020000040800f2
:206560000646204601f0aaf829468246484601f0a5f80146504600f099ff494605464046be
:020000040800f2
:2065800001f09cf800998046204601f097f80146404600f089ffd7f8c430044601991846e7
:020000040800f2
:2065a000009301f08bf8d7f8c88083463146404601f084f801465846d7f8d0a0d7f8cc903b
:020000040800f2
:2065c00000f072ff29468346484601f077f80146584600f069ff21468346504601f06ef8da
:020000040800f2
:2065e0000146584600f060ff0199c7f8c400404601f064f831468346009801f05ff8014610
:020000040800f2
:20660000584600f053ff29468346504601f056f80146584600f04aff21468346484601f0c0
:020000040800f2
:206620004df80146584600f03fff0199c7f8c800484601f043f831468346504601f03ef82a
:020000040800f2
:206640000146584600f030ff29468346009801f035f80146584600f029ff21468346404695
:020000040800f2
:2066600001f02cf80146584600f020ff0199c7f8cc00504601f022f831468246484601f08d
:020000040800f2
:206680001df80146504600f011ff29460646404601f014f80146304600f006ff2146054666
:020000040800f2
:2066a000009801f00bf80146284600f0fffe1249c7f8d0000846fff713fdfff7c7fc97f826
:020000040800f2
:2066c000c220b7f8400007eb4201013202f03f02a1f8420087f8c22090e6b2f5806f02d232
:020000040800f2
:2066e0000132fa87bbe6fff74cfdb8e6502000206fa18b3a0ad7a33bbc1f002010b5fbf792
:020000040800f2
:2067000087fc00230e4cc4e90233e3872360a3802361a3612362a382a383a384a36223637d
:020000040800f2
:20672000a363a385a386a387a4f84030fff77cfc044b1b7884f8f430012384f8043110bd3a
:020000040800f2
:20674000f81e0020a007002015494a684b8843ea0243144a1268d21a134b8a601b78052b18
:020000040800f2
:206760001dd8cb681148a3f57863db10a02ba8bfa0230068a0f5ea4030388342b8bf034631
:020000040800f2
:20678000002b0cddb3f5807fa8bf4ff48073c3f5807383fb02321b0a43ea02638b607047eb
:020000040800f2
:2067a00008200020f81f002050200020f41f00202de9f047032540f28f234b4c2269e168d3
:020000040800f2
:2067c00082fb0550c1fb0350d4e900612d0945ea0075ad1941eb201ad4e90610c2fb031011
:020000040800f2
:2067e000d4e90867414b80461b788946052bc4e9005ac4e9061063d8fff7a6ff40f2152c76
:020000040800f2
:206800003b4b3c4ab3f90430b2f90020a0689b1a394a40f69a5e12685343da179b1b62eb4f
:020000040800f2
:2068200007021b0c43ea0243da17920042ea93729900c0fb0c124d194aeb020140f26e2230
:020000040800f2
:2068400083fb022cc0fb0e2c41f65a0e12eb090248eb0c0c4ff06808a36283fb0e3ec0fb6c
:020000040800f2
:20686000083e9b1947eb0e07c4e908371b0c43ea0743c4e9005123612d0c236b45ea01458f
:020000040800f2
:20688000c4e9062c216c120c9d4242ea0c42e260c8bf2563d4e90e325b1a62ebe172174952
:020000040800f2
:2068a000e56209685b1842ebe172c4e90e323f3342f10002db0943ea42632364bde8f08740
:020000040800f2
:2068c000fff742ff40f289735146a0684a46c446c0fb03514bf20f4348f2826ec0fb032c68
:020000040800f2
:2068e0003346c0fb0e37bfe7082000205020002018030020fc1e002000200020f81f0020b5
:020000040800f2
:2069000080b5fff7fbfe0023714c724e724d2370fff728fd0028fbd02378072bf8d801a213
:020000040800f2
:2069200052f823f04569000811690008b5690008e5690008116a00081f6a00085f6a000861
:020000040800f2
:20694000876a0008654ab2f90430bbb1b2f91220a2b16349b1f900006249b1f900108f10ba
:020000040800f2
:20696000a3eba101884209db3a44904206dc5e4a126802f57a72b2f5fa5f02d90923237068
:020000040800f2
:206980000ce0627872b93b4498420bda02232370fef796fc4ff40070fbf784fd4c48fbf7dd
:020000040800f2
:2069a0007bfcb5e701232370a378002bf2d009232370efe74d4b1b68142b08dc4c4b1b6818
:020000040800f2
:2069c000b3f5a07fa4dd4b4b1b68502ba0dd03233f482370fbf760fc2b68c4e90133fff766
:020000040800f2
:2069e0008df995e7424b1a6812f1280f06db61682b685b1a40f2dc518b4289dd0423344865
:020000040800f2
:206a00002370e260fbf748fc238a013323827fe7384b1b68b3f5786f12da0523afe72f4bc6
:020000040800f2
:206a20009b8f3bb1a1682a68521a64214b439a42fff66eaf2f4b1b68002b01da06239ee787
:020000040800f2
:206a40002b4ae3681268d21a03eb6213b3f5a07fe3607ff75daf2b68636003238fe71f4bc5
:020000040800f2
:206a60005a88224b1b689a42fff652af072318482370fbf711fc2b6803f57a73636133687f
:020000040800f2
:206a8000c4e9063344e73368e2699342a269b8bfe3619342c8bfa36162692b689b1a002bc6
:020000040800f2
:206aa000fff636afd4e906329b1a042b07dc082307482370fbf7f0fb0020fbf779fe336832
:020000040800f2
:206ac000c4e906332b6803f57a73636120e700bf5020002048200020f01f0020180300204c
:020000040800f2
:206ae000cc1f0020fe1f0020d41f002034200020182000201420002000230348034a044913
:020000040800f2
:206b000000f8203bfbf71abb5020002099a800080169000810b5104b104c1b78207063709e
:020000040800f2
:206b2000fbf7fafd0e4b60801b882046a3800d4b01221b881021e3800b4b1b6823810b4b82
:020000040800f2
:206b40001b6863810a4b1b68a3810a4b1b88e381bde81040fcf72eba50200020982200203c
:020000040800f2
:206b600030110008941c002018200020142000203420002060200020f8b5324c2388002b3b
:020000040800f2
:206b80004bd00a26304c04f110076420fbf7fcfb07210120fcf7befa4ff480032b4d012062
:020000040800f2
:206ba0002b61fff7b7ff012206213846fcf770fa402301202b61fcf7bdfab4f91230b4f922
:020000040800f2
:206bc0001020db439a420cbf01230023a37528d11f4f204ea37d43b3217d3846fbf78afbe3
:020000040800f2
:206be000072120b30120fcf795fa4ff4800302202b61fff78fff3046fbf711fe0122617d87
:020000040800f2
:206c000015489140fcf744fa3046fbf725fe402301202b61fcf78efadce72046fbf712fbd7
:020000040800f2
:206c2000ace7013e16f0ff06afd1fbf7b7fb0120fcf770fa4ff4800303202b61fff76aff01
:020000040800f2
:206c4000e5e700bf941c002098220020000c014050200020af220020b022002070b5104cbe
:020000040800f2
:206c60001048a17d01f0fef8a37dc3b1637d227d218a0d4801f0f6f800250c4e627debb2ca
:020000040800f2
:206c80009a4204d8bde870400a2001f0fdb804eb43033046198b01f0e5f80135eee770bdc2
:020000040800f2
:206ca00098220020a0a80008b7a80008e7a800080c4a08b593690c4843f0080393614023b4
:020000040800f2
:206cc0000a4a1361136823f0706343f080731360faf7eefdbde80840054a06490648fbf74b
:020000040800f2
:206ce0002dba00bf00100240d4b70008000c0140eca80008796b0008c82200200c2310b536
:020000040800f2
:206d0000064c03fb0044204601f072f8044a2146bde810400244034801f0a4b8fcb70008db
:020000040800f2
:206d200043a90008f6a8000870b5054606880eb9012043e074423440802c68d014d8082c82
:020000040800f2
:206d400009d874b1631e072b0bd8dfe803f030380a3f0a0a0a43202c44d0402c46d0102cad
:020000040800f2
:206d60003cd026ea0406e2e7b4f5006f6dd010d8b4f5007f5cd0b4f5806f61d0b4f5807f22
:020000040800f2
:206d8000efd1fbf7c9fc3a4b1b68c01a6b6998421ae0b4f5804f5dd0b4f5004f61d0b4f57b
:020000040800f2
:206da000805fded1334b1a88b5f9223003e0b5f90220314b1b689a42d3da002070bdb5f9ef
:020000040800f2
:206dc00004202d4b1b689a42f7dccae7b5f906202a4befe7b5f90820284bf3e7b5f90a201a
:020000040800f2
:206de000274be7e7b5f90c20254bebe70123254ab2f9001032f9020f01338142dbb2b8bfb2
:020000040800f2
:206e00000146402bf6d1b5f90e308b42d4e701231c4ab2f9001032f9020f01338142dbb280
:020000040800f2
:206e2000b8bf0146402bf6d1b5f910308b42cbe7fbf772fc0e4b1b68c01aab699842bbe74f
:020000040800f2
:206e40000e4b1b68002bb8dd8be70c4b1b68002bb3da86e70c4b95f820201b789a42acd90d
:020000040800f2
:206e60007fe7094b95f821201b789a42a5d878e7582000206020002018200020142000205b
:020000040800f2
:206e8000342000203a1f00205020002003280ad8dfe800f0020a111881f00103c90341ea10
:020000040800f2
:206ea000c3710b4b1961704781f00103890241ea8361084bf6e781f00103490241ea436149
:020000040800f2
:206ec000054befe781f00103090241ea0361f7e70008014000100140000c014010b50022d1
:020000040800f2
:206ee000044644fa02f3d90703d50121d0b2fff7cdff0132042af4d10a4bb3f8fa00fbf7e5
:020000040800f2
:206f000043fa002244fa02f3db0703d50021d0b2fff7bcff0132042af4d1bde81040052091
:020000040800f2
:206f2000fbf732ba180300202de9f74ffbf770f8dff8d88098f80030022b42d94ff0010902
:020000040800f2
:206f4000334d0a212846fbf7d5f998f80030072b54d8002426462746dff8b8a0dff8b8b0cf
:020000040800f2
:206f6000ab8ae98a0b439bb22341da0736d4bbf840309bb3daf800300bf14006abb93046f0
:020000040800f2
:206f8000fff7d2fe48b3bbf840309b041dd5dbf85c3023eae3730193fbf7befb019b034498
:020000040800f2
:206fa000012b38bf0123caf800303046fff7bcfe30b3fbf7b1fbdaf80030c01a002808da0b
:020000040800f2
:206fc0000be04046fbf73ef9b4e7daf80030002bebd109fa04f33b439fb201260134042c3e
:020000040800f2
:206fe0000af1040a0bf12c0bbad12fb1ab8a38463b43ab82fff772ff002ea2d1fbf7cef9cb
:020000040800f2
:20700000e98a09fa04f30b43eb82e6e750200020f0240020f42400201803002030b5eff37d
:020000040800f2
:207020001085044691b072b66846fcf7f7fa85f3108840f2e93210ab03eb4404bdf9123030
:020000040800f2
:2070400034f93c0c93420cddb0ebe30f09dbc3eb031343f30f139842d4bf0020012011b001
:020000040800f2
:2070600030bd0320fbe770b50024074e074de0b2fff7d4ff214656f820200134284600f049
:020000040800f2
:20708000f1fe042cf3d170bd3cae0008fba800082de9f84f0421244800f0e4fe0025234cef
:020000040800f2
:2070a000dff88c902946234800f0dcfeb4f840308bb10026dff880b004f140070c22f0b2a8
:020000040800f2
:2070c00002fb009abaf80480b8f1000f0dd10a2000f0dafe02e0194800f0dcfe0135042de7
:020000040800f2
:2070e00004f12c04ded1bde8f88fb4f8401018ea010f0cd0fff702fe9af80620ff2a0ed0f1
:020000040800f2
:20710000b8f5804f05d3b95c584600f0abfe0136d4e718f40c5f14bfb958b95ef4e7084840
:020000040800f2
:2071200000f0a0fef3e700bf13a9000818030020fcb7000823a9000839a900082ea90008d1
:020000040800f2
:207140003fa900082de9f04f5e4f8fb0faf7b8fa3b783f2b1fd100265b4fdff8708110e0c6
:020000040800f2
:207160002846fff7cbfda3790136ff2b0cbf4046574800f077fe0c2303fb0573986800f07c
:020000040800f2
:2071800089fe0c24f5b204fb0574a388002be7d10fb0bde8f08ffaf735fbdff8388105462c
:020000040800f2
:2071a00098f800100029f3d1032806d901464a480fb0bde8f04f00f055be03ac2c22204656
:020000040800f2
:2071c00000f00efefaf77cfa3b780a2b67d00df1080b0026da465ffa86f9faf763fa50b9a7
:020000040800f2
:2071e0003a780a2a07d00bf8012b0136faf70efa032ef0d1b14609f138030deb03094ff012
:020000040800f2
:2072000000030c2209f8303c00232f49deb202fb0616b6f80490b9f1000f07d151462f48ab
:020000040800f2
:2072200000f020fe022388f80030b1e751463046019300f0a3fd019b0c2201330028e4d1c7
:020000040800f2
:20724000bdf80c30b67949ea0303ff2eadf80c30b8d0faf735fa3b782d2b17d1faf7d6f96c
:020000040800f2
:207260004ff0ff3afaf7cefa98f800300afb00f0002b8dd1b9f5804f0bd30028d2db06f178
:020000040800f2
:2072800038030deb030606f82c0c9be74ff0010ae8e719f40c5f14bfa051a05392e7faf748
:020000040800f2
:2072a00097fc2c220e4b02fb05350fcc40350fc50fcc0fc594e8070085e80700faf71cfd89
:020000040800f2
:2072c00066e700bfeb000020fcb7000842a9000847a90008ec0000204ca9000866a90008d1
:020000040800f2
:2072e0001803002010b504460146074800f0bafd032c03d90222054b1a7010bd0120a04030
:020000040800f2
:2073000080b2bde81040e9e57da90008ec0000202de9f047394b8cb05a78182a63d803f1ee
:020000040800f2
:20732000be0203f1f005ce332c4610685168083203c49a422546f7d1304e0327b046dff87b
:020000040800f2
:20734000c0902a2200210df1060000f049fd2d4811258646b6f89e3006f19e04adf80430d1
:020000040800f2
:207360000df1040c8279ff2a27d00023818839f823a08a453cd10eeb830393f8cfa093f8e4
:020000040800f2
:20738000ce30baf1080f0dd0baf1200f2ed0e35eb1f5804f0ad3002b0fdb30326a4402f8c6
:020000040800f2
:2073a0002c3c0ae0e35cb1f5804ff6d211f40c5f14bf4cf802302cf80230013d00f10c00b5
:020000040800f2
:2073c000d0d108f1c40401ad0fcd0fc40fcd0fc495e80700013f7b1c84e80700a6f12006b4
:020000040800f2
:2073e000a8f12c08add10cb0bde8f087e358cfe701330e2bbbd10023d5e700bf18030020a7
:020000040800f2
:20740000c8b80008fcb700081f4b20499a69204842f004029a614ff000420a614a6822f008
:020000040800f2
:20742000704242f080524a609a6942f010029a614ff08062c1f81028d1f8042822f47062bb
:020000040800f2
:2074400042f48072c1f804284ff000719a6942f008029a610f4a1161516821f0f00141f07e
:020000040800f2
:2074600010015160996941f0080199614ff0807313615368084923f00f0343f00103536053
:020000040800f2
:20748000064afaf75bbe00bf001002400008014008250020000c0140296f000890a90008bd
:020000040800f2
:2074a00080f0004002e000bf81f0004142001fbf5fea410392ea030f7fea226c7fea236c9f
:020000040800f2
:2074c0006ad04fea1262d2eb1363c1bfd218414048404140b8bf5b42192b88bf704710f048
:020000040800f2
:2074e000004f40f4000020f07f4018bf404211f0004f41f4000121f07f4118bf494292eaac
:020000040800f2
:20750000030f3fd0a2f1010241fa03fc10eb0c00c3f1200301fa03f100f0004302d5494218
:020000040800f2
:2075200060eb4000b0f5000f13d3b0f1807f06d340084fea310102f10102fe2a51d2b1f117
:020000040800f2
:20754000004f40ebc25008bf20f0010040ea03007047490040eb0000013a28bfb0f5000f99
:020000040800f2
:20756000edd2b0fa80fcacf1080cb2eb0c0200fa0cf0aabf00ebc25052421843bcbfd040f4
:020000040800f2
:207580001843704792f0000f81f4000106bf80f400000132013bb5e74fea41037fea226c1a
:020000040800f2
:2075a00018bf7fea236c21d092ea030f04d092f0000f08bf0846704790ea010f1cbf0020c7
:020000040800f2
:2075c000704712f07f4f04d1400028bf40f00040704712f100723cbf00f50000704700f0f5
:020000040800f2
:2075e000004343f0fe4040f4000070477fea226216bf08467fea23630146420206bf5fea54
:020000040800f2
:20760000412390ea010f40f4800070474ff0000304e000bf10f0004348bf40425fea000c0b
:020000040800f2
:2076200008bf704743f0964301464ff000001ce050ea010208bf70474ff000030ae000bf98
:020000040800f2
:2076400050ea010208bf704711f0004302d5404261eb41015fea010c02bf844601460020fc
:020000040800f2
:2076600043f0b64308bfa3f18053a3f50003bcfa8cf2083aa3ebc25310db01fa02fc634471
:020000040800f2
:2076800000fa02fcc2f12002bcf1004f20fa02f243eb020008bf20f00100704702f120023f
:020000040800f2
:2076a00001fa02fcc2f1200250ea4c0021fa02f243eb020008bf20eadc7070474ff0ff0c19
:020000040800f2
:2076c0001cead0521ebf1cead15392ea0c0f93ea0c0f6fd01a4480ea010c400218bf5fead6
:020000040800f2
:2076e00041211ed04ff0006343ea501043ea5111a0fb01310cf00040b1f5000f3ebf490078
:020000040800f2
:2077000041ead3715b0040ea010062f17f02fd2a1dd8b3f1004f40ebc25008bf20f001007c
:020000040800f2
:20772000704790f0000f0cf0004c08bf49024cea502040ea51207f3ac2bfd2f1ff0340ea3f
:020000040800f2
:20774000c250704740f400004ff00003013a5ddc12f1190fdcbf00f000407047c2f1000214
:020000040800f2
:20776000410021fa02f1c2f1200200fa02fc5fea310040f1000053ea4c0308bf20eadc7099
:020000040800f2
:20778000704792f0000f00f0004c02bf400010f4000f013af9d040ea0c0093f0000f01f094
:020000040800f2
:2077a000004c02bf490011f4000f013bf9d041ea0c018fe70cead15392ea0c0f18bf93eaa7
:020000040800f2
:2077c0000c0f0ad030f0004c18bf31f0004cd8d180ea010000f00040704790f0000f17bfa4
:020000040800f2
:2077e00090f0004f084691f0000f91f0004f14d092ea0c0f01d142020fd193ea0c0f03d12f
:020000040800f2
:207800004b0218bf084608d180ea010000f0004040f0fe4040f40000704740f0fe4040f487
:020000040800f2
:20782000400070474ff0ff0c1cead0521ebf1cead15392ea0c0f93ea0c0f69d0a2eb0302de
:020000040800f2
:2078400080ea010c49024fea402037d04ff0805343ea111143ea10130cf000408b4238bf15
:020000040800f2
:207860005b0042f17d024ff4000c8b4224bf5b1a40ea0c00b3eb510f24bfa3eb510340ea64
:020000040800f2
:207880005c00b3eb910f24bfa3eb910340ea9c00b3ebd10f24bfa3ebd10340eadc001b019e
:020000040800f2
:2078a00018bf5fea1c1ce0d1fd2a3ff650af8b4240ebc25008bf20f0010070470cf0004c83
:020000040800f2
:2078c0004cea50207f32c2bfd2f1ff0340eac250704740f400004ff00003013a37e792f0c7
:020000040800f2
:2078e000000f00f0004c02bf400010f4000f013af9d040ea0c0093f0000f01f0004c02bf5f
:020000040800f2
:20790000490011f4000f013bf9d041ea0c0195e70cead15392ea0c0f08d142027ff47dafe4
:020000040800f2
:2079200093ea0c0f7ff470af084676e793ea0c0f04d14b023ff44caf08466ee730f0004c7b
:020000040800f2
:2079400018bf31f0004ccad130f000427ff45caf31f000437ff43caf5fe700bf4ff0ff3c27
:020000040800f2
:2079600006e000bf4ff0010c02e000bf4ff0010c4df804cd4fea40024fea41037fea226c24
:020000040800f2
:2079800018bf7fea236c11d001b052ea530c18bf90ea010f58bfb2eb030088bfc81738bfb6
:020000040800f2
:2079a0006feae17018bf40f0010070477fea226c02d15fea402c05d17fea236ce4d15fea13
:020000040800f2
:2079c000412ce1d05df8040b704700bf844608466146ffe70fb5fff7c9ff002848bf10f158
:020000040800f2
:2079e000000f0fbd4df808edfff7f4ff0cbf012000205df808fb00bf4df808edfff7eaff4d
:020000040800f2
:207a000034bf012000205df808fb00bf4df808edfff7e0ff94bf012000205df808fb00bf61
:020000040800f2
:207a20004df808edfff7d2ff94bf012000205df808fb00bf4df808edfff7c8ff34bf01208f
:020000040800f2
:207a400000205df808fb00bf4fea4002b2f1fe4f0fd34ff09e03b3eb12620dd94fea00236e
:020000040800f2
:207a600043f0004310f0004f23fa02f018bf404270474ff00000704712f1610f01d14202a3
:020000040800f2
:207a800005d110f0004008bf6ff0004070474ff00000704753b94ab9002908bf00281cbfbb
:020000040800f2
:207aa0004ff0ff314ff0ff3000f066b9adf1080c6de904ce00f006f8ddf804e0dde902236e
:020000040800f2
:207ac00004b070472de9f047089d0e4604468e46002b4cd18a429446b2fa82f362d953b189
:020000040800f2
:207ae00002fa03fcc3f1200201fa03fe20fa02f242ea0e0e9c404fea1c47befbf7f11ffa31
:020000040800f2
:207b00008cf607fb11ee01fb06f0220c42ea0e4290420ad91ceb020201f1ff3e80f00e8158
:020000040800f2
:207b2000904240f20b8102396244121ab2fbf7f007fb102200fb06f6a4b244ea0244a64237
:020000040800f2
:207b40000ad91ceb040400f1ff3280f0f980a64240f2f6806444023840ea01400021a41b6b
:020000040800f2
:207b60001db1dc400023c5e90043bde8f0878b4205d90db1c5e9000100210846f5e7b3fadb
:020000040800f2
:207b800083f1002942d1b34202d3824200f2ee80841a66eb030201209646002de5d0c5e9c6
:020000040800f2
:207ba000004ee2e7002b40f08c80881a0121170c96b2b0fbf7fe07fb1e00220c42ea0042bc
:020000040800f2
:207bc00006fb0ef0904208d91ceb02020ef1ff3802d2904200f2cc80c646121ab2fbf7f002
:020000040800f2
:207be00007fb102200fb06f6a4b244ea0244a64208d91ceb040400f1ff3202d2a64200f2e8
:020000040800f2
:207c0000b2801046a41b40ea0e40a9e7c1f120078b4022fa07fc4cea030c26fa07fa4feab3
:020000040800f2
:207c20001c48bafbf8fe06fa01f308fb1eaa1ffa8cf620fa07f400fa01f90efb06f023436d
:020000040800f2
:207c40001c0c44ea0a44a04202fa01f20bd91ceb04040ef1ff3a80f08480a04240f28180fb
:020000040800f2
:207c6000aef1020e6444241a98b2b4fbf8f308fb134403fb06f640ea0444a64208d91cebf5
:020000040800f2
:207c8000040403f1ff3068d2a64266d9023b644443ea0e40a41ba0fb02e6b4427346b04611
:020000040800f2
:207ca00052d34fd05db1b9eb030264eb080404fa07f722fa01f31f43cc40c5e900740021b1
:020000040800f2
:207cc00053e702fa03fcc3f12000c1404fea1c47b1fbf7fe07fb1e1124fa00f09e403043cd
:020000040800f2
:207ce000020c1ffa8cf642ea01420efb06f1914204fa03f409d91ceb02020ef1ff382ed281
:020000040800f2
:207d000091422cd9aef1020e6244521ab2fbf7f107fb112280b240ea024001fb06f28242aa
:020000040800f2
:207d200008d91ceb000001f1ff3814d2824212d902396044801a41ea0e413ae77146f4e6f8
:020000040800f2
:207d4000104609e7f145add2beeb020366eb0c060138b046a6e74146ece7034698e7c6462d
:020000040800f2
:207d6000d3e7d6467fe7644402384be7084614e7aef1020e624430e7704700bf10f8012b54
:020000040800f2
:207d800011f8013b012a28bf9a42f7d0d01a70470a44914200f1ff3300d1704710b511f8ae
:020000040800f2
:207da000014b914203f8014ff9d110bd884210b501eb020402d98442234607d8431ea14214
:020000040800f2
:207dc00008d011f8012b03f8012ff8e7014602448a4200d110bd13f8014d02f8014df7e716
:020000040800f2
:207de00003460244934200d1704703f8011bf9e7034613f8012b002afbd1181a0138704708
:020000040800f2
:207e000070b500260d4d0e4c641ba410a6420bd10c4b0bb1aff3008000260b4d0b4c641be3
:020000040800f2
:207e2000a410a64205d170bd55f8043b98470136ece755f8043b98470136f2e7d8a2000831
:020000040800f2
:207e4000d8a2000800000000d8a20008dca20008024bc01a024b1860704700bf080000002e
:020000040800f2
:207e6000302700200fb407b5064b04aa52f8041b1868019200f0e4f803b05df804eb04b01a
:020000040800f2
:207e8000704700bf38ae0008014b196801f09dbc38ae0008f8b50e4b06461d68ab789b07dd
:020000040800f2
:207ea00012d56f6816f8014b29462cb90a20b847002805db204609e02046b8470028f1da7e
:020000040800f2
:207ec000ab7843f00403ab704ff0ff30f8bd00bf38ae00082de9f0470746884616464ff057
:020000040800f2
:207ee000000ac3f137095ffa89f903f01f05384641462a465346fff7cdfdd4b23a46434635
:020000040800f2
:207f0000092c84bf4c44e4b2aa4204f1300473eb0a030746884606f8014be8d23046bde809
:020000040800f2
:207f2000f08700002de9f04101260746b24201dcbde8f0813b461f4613f8014b002cf7d0f8
:020000040800f2
:207f4000252cf8d11d780237252df3d000239c461c46dff8e8801f2c27d8a5f1200ebef1c1
:020000040800f2
:207f6000100f06d828fa0efe1ef0010f53d12e2d3cd02e2d27d8242d33d02a2d36d0bcf175
:020000040800f2
:207f8000000fd5d0b445d1d145f02007a7f1650cbcf1020f0b6801d9612f42d1073323f032
:020000040800f2
:207fa000070308330b600136bfe77f2cdfd96c2d23d01dd8682d27d06a2d01d04c2dded134
:020000040800f2
:207fc00044f4207408e0a5f1300ebef1090feed80a2404fb03e3202417f8015b002dbad112
:020000040800f2
:207fe000cde7bcf1000f18d0b34218d00023f3e7742df1d07a2defd0c1e7250648bf44f475
:020000040800f2
:20800000007444f08004e7e7e50548bf44f4007444f48074e0e70024dee79c46e6e76325b6
:020000040800f2
:20802000b2e7692d02d007d8632d03d0250601d5a405b3d40433b5e7732df6e789280100ca
:020000040800f2
:208040002de9f04f837895b09c07cde908124768039015d50b4600250d92187890b12528b9
:020000040800f2
:2080600014d0013306930399b847002805f1010580f2fb83039b039a9b7843f00403937015
:020000040800f2
:208080004ff0ff35284615b0bde8f08f93f801809a1cb8f1250f0692e5d000242646a146b3
:020000040800f2
:2080a000a246baf11f0f23d8a8f12003102b23d8dfe803f01522221b2222220b22222213fa
:020000040800f2
:2080c0002218222209004af0010a069b13f8018b0693b8f1000fe4d11ce04af0020a4af01a
:020000040800f2
:2080e000040af2e74af0080aefe74af0100aece7baf17f0f00f2ef80b8f12e0f00f0cc8094
:020000040800f2
:2081000000f2a580b8f1240f00f0cd80b8f12a0f00f0ac8034b1099b224608980da90d934a
:020000040800f2
:20812000fff700ff002e48f02003b8bf2af0400a0593a3f16503bcbf00261ffa8afa022be7
:020000040800f2
:2081400004d948f02003612b40f0a4826fea080808f0200307930d9b073323f0070303f1f4
:020000040800f2
:2081600008020d92059ad3e90001612a0af0400340f0e080002b079b0eaa009314bf33463e
:020000040800f2
:208180004ff0ff3301f08afa431cdbb20493702306464ff00108ddf838b04af4c05a0593a2
:020000040800f2
:2081a0000bf10903122b0ed90bf16303c62b40f2fd8340f2ce720bf2e73393428cbf4ff0a6
:020000040800f2
:2081c00004084ff003089df83c20d00700f1e1801af0020f40f0df80caf380035b0112f0e7
:020000040800f2
:2081e0000c0f00f0e380002b0cbf032404244c4511da1af0080fa9eb04040dd12c44202005
:020000040800f2
:2082000003990493b847002805f10105fff632afac42049bf3d100243bb118460399b847d8
:020000040800f2
:20822000002805f10105fff625af9df83c30aa4e13f0080fa94b08bf1e46b146c84619f809
:020000040800f2
:20824000010b002840f0a980ae1bb04486e1a8f13003092b3fd80a221af0400f12bf02fb03
:020000040800f2
:20826000063602fb09394af0200a2ee7002c7ff42caf0d9a1af0400f52f8043b0d9201d097
:020000040800f2
:208280001e4622e7002ba7bf99464af0200ac3f100094af0280a18e71af0400f7ff4f2ae09
:020000040800f2
:2082a0004af0400a11e7002c3fd0099b1af040080cbf4a46324608980da90d93fff732fe22
:020000040800f2
:2082c0000d9b1a1d0d92b8f1000f01d01e68fce6d3f80090f9e6b8f16c0f16d00cd8b8f15e
:020000040800f2
:2082e000680f1ad0b8f16a0f03d0b8f14c0f7ff411af4af4207ae8e6b8f1740f3ff4e5ae59
:020000040800f2
:20830000b8f17a0f3ff4e1ae04e71af0800f18bf4af4007a4af0800ad7e61af4807f18bff1
:020000040800f2
:208320004af4007a4af4807acfe626464c46b246b146cae6002b059b08bf0626652b14d1c8
:020000040800f2
:2083400000221446731cdbb24af4805a112b28bf1123cde900240eaa00f000fcc3b24ff0e4
:020000040800f2
:208360000208ddf838b004931ae7059b662b05d13446012211234af4005ae7e700224ff0ff
:020000040800f2
:20838000650cf3b2012b38bf01231446cdf814c0dce72d2323e72b2321e7079b0399c01a02
:020000040800f2
:2083a000c0b2b8470028bff649af63e61af4405f1dd1002e08bf0126049a50326a44133a5c
:020000040800f2
:2083c000049919b112f8011d30297bd01af0100f049a18bf32461bf1040f78dbb34576da9a
:020000040800f2
:2083e0005a454af4005a74dd0bf10106961b1af400520a9274d02beaeb74013403b101346f
:020000040800f2
:20840000002e74d0721c1444a145d4bf0024a9eb04041af0090f03d12c44a5426cd100241d
:020000040800f2
:208420003bb118460399b847002805f10105fff621ae1af4006f11d030200399b8470028fe
:020000040800f2
:20844000fff618ae079b0399c3f1780000f0f800b847002805f10205fff60cae1af0080f1b
:020000040800f2
:2084600003d12c44a54251d100240a9b002b7ad02beaeb79abeb09027642049b09f1ff39ce
:020000040800f2
:20848000934285bf0eabd318302058794e45059205f1010842dc0399b847059a002802f162
:020000040800f2
:2084a0000102fff6e7adb9f1ff3f09d12e2003990592b8470028fff6ddad059a05f10208a8
:020000040800f2
:2084c0004546dae704990139c9b2049178e7561e8de700268be700bfcfaa0008cbaa0008cd
:020000040800f2
:2084e0001af4006f14bf05240324444486e71af0100f18bf013487e7202003990b93b847cb
:020000040800f2
:2085000000280b9b05f1010587dab3e530200399b847002805f10105a4daabe5cb450ad190
:020000040800f2
:208520009df83d30352b1cd805d19df83c3013f0100f08bf31200399b8470028fff69aadd5
:020000040800f2
:208540001af0100f0ad0b9f1ff3f07d12e20039905f10208b8470028fff68cad4546444406
:020000040800f2
:2085600020e23120e7e79df83d00039931281ebf9df83c3023f010038df83c30b8470028f7
:020000040800f2
:20858000fff678ad002e67dd2e200399b8470028fff670ad4ff00109049b03994b45c5bf94
:020000040800f2
:2085a0000eab4b4430205879b8470028ca46fff661ad09f101094e45eeda02355544059b49
:020000040800f2
:2085c000079a0399981ac0b2b8470028fff652adbbf1000f04db4cd19df83c30db0648d569
:020000040800f2
:2085e0002d20cbf1000b0399b8470028fff642adb8f1040f3fd14ff47a78bbfbf8f606f124
:020000040800f2
:2086000030000399c0b2b847002805f10305fff631ad08fb16bb4ff06408bbfbf8f606f10a
:020000040800f2
:2086200030000399c0b2b847002805f10105fff621ad08fb16bb4ff00a08bbfbf8f606f156
:020000040800f2
:2086400030000399c0b2b847002805f10105fff611ad08fb16bb16e01af0100f01d101350b
:020000040800f2
:20866000ade72e200399b847002805f10205a6da00e52b20b7e7b8f1030f05f10205cad0b8
:020000040800f2
:20868000b8f1010fd7d10bf13000039905f10108c0b25fe7a8f16303122b00f2d180dfe8b4
:020000040800f2
:2086a00013f013005300cf00cf00cf00cf005300cf00cf00cf00cf00cf00e700c900cf0038
:020000040800f2
:2086c000cf002800cf00a70001260d9b0eac1a1d1b680d928df838301af0080f2bd0a0465c
:020000040800f2
:2086e00004eb060ad04528d12c1ba044a9eb060434e70d9b1a1d0d921c68ae4b002c08bf9b
:020000040800f2
:208700001c461af0400f14bf31464ff0ff31204600f0b8ff0646dfe720200399b8470028c3
:020000040800f2
:20872000fff6a8ac08f1ff384645f5d34d44a5eb0805c146d3e7c846f6e7039918f8010bdb
:020000040800f2
:20874000b8470028ceda95e41af0800f0d9b3dd01af4007f35d0073323f0070303f108029c
:020000040800f2
:208760000d92d3e90001002904da404261eb41014af4806a2af0100b50ea01031ffa8bfb4c
:020000040800f2
:2087800005d11af0400f02d0002e00f08b800a230df1380a5246fff79dfba0eb0a0a1bf072
:020000040800f2
:2087a000400f00f081802bf0010356459bb240f38580b8f1000f02d12bf011039bb23446b9
:020000040800f2
:2087c00074e01a1d18680d92c117cce71a1d1af4807f19680d9201d10846f5e71af4007f77
:020000040800f2
:2087e00015bf48b208b241f3c01141f3c031bae70a232af0100a1ffa8afa1af080040d9af3
:020000040800f2
:208800003ad01af4007115bf0732101d22f007020d900fbf106802f108010d91d2e9000141
:020000040800f2
:2088200050ea010235d02af0060a1ffa8afb0df1380aafe710234ff078084af0100adce74f
:020000040800f2
:20884000059b782b04d1c8f1780343f01003d4e725200399b8470028fff60cac40460399f4
:020000040800f2
:20886000b8470028fff606ac0235069bfff7f5bb08234ff00008c0e7111d0d911af48071c8
:020000040800f2
:208880001068cdd01af400711abf2146c0b280b2c6e72af0160b1af0400f1ffa8bfbc6d0ea
:020000040800f2
:2088a000002ec4d1b2467ae754465b4613f0100216d0b8f1000f03d1013402e05446f5e74d
:020000040800f2
:2088c000023413f0080f22d113f0010f06d0a14531dda9eb040404eb0a064c46a34610e072
:020000040800f2
:2088e00040f206410b42ecd0e6e720200399cde90432b8470028fff6bdabdde904320bf1e5
:020000040800f2
:20890000010bd945f1dc2c1b04eb0b055c46a2b130200399b8470028fff6acabb8f1000f0e
:020000040800f2
:208920002ed0404603990235b8470028fff6a2aba8462e4419e05646d0e740f206421342fc
:020000040800f2
:20894000f6d013f0020f14bf2b20202013f4806f18bf2d2003990135e6e730200399b8473b
:020000040800f2
:20896000002808f10108fff685aba6eb08039a45f3db55460eae2db9d044a9eb0404ede5a0
:020000040800f2
:208980000135d5e7013d0399705db8470028f2dafff770bb20200399b847002805f101052b
:020000040800f2
:2089a000fff668ab631b002bf4dc5ee74ff0020809e400bfd3aa00082de9f04f87b00618cd
:020000040800f2
:2089c000994602ab41eb010400931546d2e9002330462146ddf844b000f00efc04ab00932c
:020000040800f2
:2089e0000746d5e9022388463046214600f004fcdde90263841951eb03064ff00002d5e9a0
:020000040800f2
:208a0000000128bf0122049ba9f1410ad218059b43f10003381848eb0101b84271eb080122
:020000040800f2
:208a200038bf0120d5e902c128bf002014eb0c0c46eb010110eb0c0041f10001a04271ebd4
:020000040800f2
:208a4000060c34bf4ff0010c4ff0000ccde904231ceb020243f10003cdf800a000f0e7fb24
:020000040800f2
:208a6000109bc3e90001129b012bdde9042329d1d5e90201d5e900c5201a66eb0101674561
:020000040800f2
:208a800078eb050534bf01250025401b61f10001844276eb010534bf01250025cdf800a0ad
:020000040800f2
:208aa000521b63f1000300f0c2fbdde90423cbe9000120463146cdf800a000f0b8fb07b007
:020000040800f2
:208ac000bde8f08f17eb070e48eb080c201946eb0601be457ceb080834bf01270027c71907
:020000040800f2
:208ae00041f10008d5e9000186457ceb010c38bf0120d5e9021528bf0020381a68f1000c93
:020000040800f2
:208b0000401a6ceb050192185b41a74278eb060534bf01250025521943f10003874278ebf5
:020000040800f2
:208b2000010834bf01250025521ba9f140050095b7e700001fb502ab0093074a4ff0cc33cc
:020000040800f2
:208b400000f05afbdde90201c00840ea4170c90805b05df804fb00bfcdcccccc2de9f04f45
:020000040800f2
:208b60009bb00a939df89030044605920b93080dc1f31303c1f30a52c90f07917ab954ea69
:020000040800f2
:208b8000030179d13023012705994b71079b0a6043f002030b7138461bb0bde8f08f40f253
:020000040800f2
:208ba000ff718a420ad12343079b059a14bf43f0080343f0040300271371ece7a2f2354a1b
:020000040800f2
:208bc00043f4801504f001024fea85082343089248ea94784fea840652d140f2fe731842eb
:020000040800f2
:208be0000cbf01270027baf1000fc0f2b380504600f0e8f9baf1030fc8bf0138049000f054
:020000040800f2
:208c0000edf9049b7c30a3eb0a0a824416a9184600f076fa12ab019310ab204629460093ca
:020000040800f2
:208c20000297534616aafff7c7fe049b0446152b0d4600f28b8014aba64a009330464ff017
:020000040800f2
:208c4000cc33414600f0d8fadde9109a149b159a9b0843ea827303eb8303b34212d1414666
:020000040800f2
:208c6000304600f0c3f9049b83428cbf4ff000084ff00108002717e01d46dff85ca2a1e7b6
:020000040800f2
:208c80000127b0e7089b002b50d1013e48f1ff31f01b61f1000100f0a9f9049bddf820807a
:020000040800f2
:208ca00083428cbf002701270b9b002b40f0c280ddf828b000264ff00a0a06960996dde9eb
:020000040800f2
:208cc0001001fff737ff129bcde90c01184613990e93fff72fff0c9b0d9a98420b469341cb
:020000040800f2
:208ce00081460f9180f0c08020462946fff722ff0afb09f30e9a002e14bf4ff0000808f088
:020000040800f2
:208d00000108934214bf002707f001070c9b0afb104610930d9b0446cde911390f9b0d46e8
:020000040800f2
:208d20001393069bf6b201330693c8e7b01c48f1000100f05bf9049b83428cbf002001208e
:020000040800f2
:208d4000b9eb00006af10002cde910024ff000084746a9e7caf1000b584600f039f9baf1b5
:020000040800f2
:208d6000ff3facbf8146a0f10109abeb090b0aeb09035846049300f031f916a9a0f17d0a17
:020000040800f2
:208d8000584600f04bf912ab0193a9eb0a0a10ab2046294600930297534616aafff70cfef3
:020000040800f2
:208da000b9f1010f04460d460ed8089b13b94ff0010879e7109b119a013b42f1ff324ff02a
:020000040800f2
:208dc0000108cde9103255e7b9f13e0fbed84ff0ff33a9f1200003fa09f203fa00f0c9f1ff
:020000040800f2
:208de000200123fa01f102430a4303fa09f328ea020826ea030656ea08060cbf4ff0010822
:020000040800f2
:208e00004ff0000836e700fb02f6a1fb0012013332448c4275eb0206f5d2049addf828b05b
:020000040800f2
:208e20001344259a1344012bb8bf01239b45a8bf9b463fe70a21002201230846e9e70afb1c
:020000040800f2
:208e400003f0a2fb0a2301310344944275eb0300f5d259450cddbbf1000f02d154ea050381
:020000040800f2
:208e600006d0012309933fe70a2200230121ece7002f33d04ff00a0a129b139918460d9316
:020000040800f2
:208e8000fff758fe0afb00f20d9b81469a420c9124d1dde91001fff74dfe0e900d912046f8
:020000040800f2
:208ea0002946fff747fe0d9b002e14bf4ff0000808f00108cde911390c9b0afb104613936f
:020000040800f2
:208ec000069b0e9a013304460d46f6b210920693d2e700bfcdccccccccfbffffb8f1000f6f
:020000040800f2
:208ee00005d0052e03d104f001060436f6b2069bddf810809844099b53b9dde912239d424d
:020000040800f2
:208f000008bf944204d1089b002b47d1002f45d0042e94bf002601260a2230194ff000032c
:020000040800f2
:208f20004ff00107144645f10001904271eb030536d2e6b1bb451ada0b9b63b1259a08eb24
:020000040800f2
:208f40000703ddf828b0134423eae3739b45a8bf9b465f450bdd05304ff00a024ff000032a
:020000040800f2
:208f600041f10001fef796fd08f10108013f5f45a8bf5f464ff000093fb20ffa88f8b84486
:020000040800f2
:208f8000059b08f1ff3607f105089844b9450edb059b1a461e60079b1371fce50126bbe7ed
:020000040800f2
:208fa00004fb03f5a2fb042301372b44bde70a220023fef76ffd303208f8012d09f1010967
:020000040800f2
:208fc000e4e700bf014b5843800c704741340100014b5843000d7047fb2e0b00024b5843a0
:020000040800f2
:208fe000c00c0130704700bf4f93120070b503464ff0cc3600204ff03335074a06fb03f44b
:020000040800f2
:2090000002fb0144a3fb023121449d4275eb010401d30130f2e770bdcdcccccc1a232de905
:020000040800f2
:20902000f04fb0fbf3fb03fb1b03344e04460d4689b006eb0b1753b9d7e90023c1e9002315
:020000040800f2
:20904000d7e90201c5e9020109b0bde8f08f06ebc303d3e9348904ab0093d7e902234046e2
:020000040800f2
:20906000494600f0c9f806ab0093d7e90023824603914046494600f0bff8dde9067280466d
:020000040800f2
:20908000039817eb0a0752eb00094ff0000328bf012333b1049b059a013342f10002cde94e
:020000040800f2
:2090a000043220460391fff799ff82461a2000fb0bf0fff793ffaaeb000a3a464b4640463c
:020000040800f2
:2090c0000399cdf800a000f0b2f8230906eb8306640004f01e03d6f8a041dc4004f0030410
:020000040800f2
:2090e000241841f10001c5e90041dde9042338464946cdf800a000f09af8a3e700b90008e6
:020000040800f2
:209100002de9f04f1a2700f11905b5fbf7f56f43dff8e0802b018bb008f5fc7b05933b1a5d
:020000040800f2
:2091200004460e460beb05150ad1d5e90023c1e90023d5e90201c6e902010bb0bde8f08fa6
:020000040800f2
:2091400008ebc303d3e93423cde90223dde9020106ab0093d5e9022300f04ef882468946ab
:020000040800f2
:20916000059b08a95bf803206b68013a63f100030091dde9020100f03ff8dde9085215eb22
:020000040800f2
:209180000a0552eb09094ff0000328bf0123834633b1069b079a013342f10002cde90632de
:020000040800f2
:2091a00038460291fff71aff07462046fff716ff3f1a2a464b4658460299009700f037f888
:020000040800f2
:2091c000230908eb8308640004f01e03d8f8e842dc4004f003040134241841f10001c6e908
:020000040800f2
:2091e0000041dde9062328464946009700f01ff8a1e700bf00b90008f0b50f460446a0fbbd
:020000040800f2
:209200000201a7fb02524919a3fb0445a7fb037342f10002611845f10004d219059e43f14a
:020000040800f2
:209220000003121943f10003c6e90023f0bdf0b5059cc4f14007c4f1200602fa06f6a4f1a0
:020000040800f2
:209240002005bb4022fa05f53343c4f120062b4301fa06f6a4f12005e04021fa05f53043c0
:020000040800f2
:20926000ba402843e14010431943f0bd20f00042b2f1ff4f70b50346044610d3002807da25
:020000040800f2
:2092800000f0def920b12046bde8704000f0f2b921462046fef70af90446204670bd002a14
:020000040800f2
:2092a000fbd00028f0db10f0ff4127d0c2150024192526464ff08071c3f31603a2f17f0003
:020000040800f2
:2092c00043f40003d20758bf5b0040105b0072189a42cfbf1a46561864189a1a013d4feaf5
:020000040800f2
:2092e00042034fea5101f2d112b1013424f00104641004f17c5404ebc054cee75b00180264
:020000040800f2
:209300000a4601f10101f9d55242d0e720f00042b2f17e5ff8b5054607d1002800f335817d
:020000040800f2
:209320009b499c48fef7c2f8f8bd03d9bde8f84000f0a0b9b2f17c5f59d2b2f10c5f02d86e
:020000040800f2
:2093400095499648eee70146fef7b8f904469449fef7b4f99349fef7a9f82146fef7aef951
:020000040800f2
:209360009149fef7a1f82146fef7a8f98f49fef79df82146fef7a2f98d49fef795f8214670
:020000040800f2
:20938000fef79cf98b49fef791f82146fef796f9894906462046fef791f98849fef784f8c1
:020000040800f2
:2093a0002146fef78bf98649fef780f82146fef785f98449fef778f82146fef77ff94ff072
:020000040800f2
:2093c0007e51fef773f801463046fef72bfa2946fef774f901467048fef766f801462846af
:020000040800f2
:2093e000fef762f801466d48fef75ef89ce700285bda4ff07e51fef759f84ff07c51fef7a2
:020000040800f2
:209400005df90446fff732ff654905462046fef755f96449fef74af82146fef74ff96249b0
:020000040800f2
:20942000fef742f82146fef749f96049fef73ef82146fef743f95e49fef736f82146fef7cd
:020000040800f2
:209440003df95c49fef732f82146fef737f95a4906462046fef732f95849fef725f82146f7
:020000040800f2
:20946000fef72cf95649fef721f82146fef726f95449fef719f82146fef720f94ff07e5184
:020000040800f2
:20948000fef714f801463046fef7ccf92946fef715f94149fef708f82946fef707f80146b9
:020000040800f2
:2094a000fef704f801463b489ee701464ff07e50fdf7faff4ff07c51fef700f90446fff7f1
:020000040800f2
:2094c000d5fe3749054620f47f662046fef7f6f83449fdf7ebff2146fef7f0f83249fdf79e
:020000040800f2
:2094e000e3ff2146fef7eaf83049fdf7dfff2146fef7e4f82e49fdf7d7ff2146fef7def856
:020000040800f2
:209500002c49fdf7d3ff2146fef7d8f82a4907462046fef7d3f82949fdf7c6ff2146fef777
:020000040800f2
:20952000cdf82749fdf7c2ff2146fef7c7f82549fdf7baff2146fef7c1f84ff07e51fdf7f4
:020000040800f2
:20954000b5ff01463846fef76df92946fef7b6f826f00f06074631463046fef7aff80146dd
:020000040800f2
:209560002046fdf7a1ff314604462846fdf79eff01462046fef756f901463846fdf796fff2
:020000040800f2
:209580003146fdf793ff0146cce60020cce600bf68212234da0f49406821a233da0fc93fa4
:020000040800f2
:2095a00008ef1138047f4f3a4611243da80a4e3e90b0a63eabaa2a3e2ec69d3d6133303fb7
:020000040800f2
:2095c0002d57014039d1194007b51c4a20f00043934206d80022002103b05df804eb00f011
:020000040800f2
:2095e00083b9b3f1ff4f04d303b05df804eb00f041b8694600f0eaf900f0030001280ad00e
:020000040800f2
:2096000002280dd0a0b901220199009800f06cf903b05df804fb0199009800f0ebf8f7e756
:020000040800f2
:2096200001220199009800f05ff900f10040efe70199009800f0def8f7e700bfd80f493f82
:020000040800f2
:2096400030f000400dd0a0f50003b3f1fe4f0ad3074b421e9a4208d9a0f1ff4358425841f2
:020000040800f2
:20966000704702207047042070470320704700bffeff7f0008b5fff7e3ff014808bd00bf08
:020000040800f2
:209680000000c07f024610b501448a42134603d01c780132002cf8d1181a10bd2de9f04f31
:020000040800f2
:2096a00004460d46274618460b46c1f30a512646c5f3130441ea070525435ad130214ff04d
:020000040800f2
:2096c000000c5171db0f002813715bdb0c285bdc0125c0f10d01890001f1ff39a1f1210e2c
:020000040800f2
:2096e000c1f1210825fa08f805fa0efe05fa09f54eea080e15eb05084eeb0e09d8f1000be9
:020000040800f2
:2097000069eb490a18f1ff3849f1ff3908ea070809ea040945457eeb090910dbc1f1200924
:020000040800f2
:20972000b1f1200804fa09f927fa01f141ea09015cbf44fa08f841ea0801c90709d57f1944
:020000040800f2
:209740003e4644eb0e04b4f5801fa2bf51790131517106ea0b0604ea0a04bcf5806f18d157
:020000040800f2
:20976000264313d043f008031371c2f800c0bde8f08f21b131255571a1f2ff3ca2e73025a3
:020000040800f2
:209780000121f8e70020e8e70d20e6e743f00403eae70d219df82450571dc5f1570506f021
:020000040800f2
:2097a0000f03360946ea0476241123b9884204da0139f4d1d9e7092b05dc30338842b8bf7d
:020000040800f2
:2097c00008467b54f4e72b44f8e738b58b780d469b0709d5c4b220464b689847002806da0a
:020000040800f2
:2097e000ab7843f00403ab704ff0ff3038bd2046fce700002de9f04120f00045b5f1485f5c
:020000040800f2
:20980000064688465bd30146fdf758ff4ff07c510446fdf753ff2b4907462046fdf74eff6a
:020000040800f2
:209820002949fdf743fe2146fdf748ff2749fdf73bfe2146fdf742ff2549fdf737fe2146a8
:020000040800f2
:20984000fdf73cff2349fdf72ffe2146fdf736ff2149fdf72bfe2146fdf730ff2146fdf750
:020000040800f2
:209860002dff414604463046fdf728ff01462046fdf71afe194b04469d420ad8014638466d
:020000040800f2
:20988000fdf712fe01464ff07e50fdf70dfebde8f081134b4ff07e509d428cbf114d05f172
:020000040800f2
:2098a0007f452946fdf700fe294606463846fdf7fbfd2146fdf7f8fd01463046e5e74ff046
:020000040800f2
:2098c0007e50e4e74ed747adf6740f317cf29334010dd037610bb63aabaa2a3d9999993ec1
:020000040800f2
:2098e0000000483f0000903e2de9f84320f00043b3f1485f04460f46914634d30146fdf76c
:020000040800f2
:20990000ddfe054601462046fdf7d8fe284906462846fdf7d3fe2749fdf7c6fd2946fdf730
:020000040800f2
:20992000cdfe2549fdf7c2fd2946fdf7c7fe2349fdf7bafd2946fdf7c1fe2149fdf7b6fdc9
:020000040800f2
:209940008046b9f1000f11d101462846fdf7b6fe1c49fdf7a9fd3146fdf7b0fe0146204684
:020000040800f2
:20996000fdf7a4fd04462046bde8f8834ff07c513846fdf7a3fe414681463046fdf79efe0f
:020000040800f2
:2099800001464846fdf790fd2946fdf797fe3946fdf78afd0c4905463046fdf78ffe0146a1
:020000040800f2
:2099a0002846fdf781fd01462046fdf77dfdd9e7d3c92e2f342fd7321bef3836010d503978
:020000040800f2
:2099c0008988083cabaa2a3eabaa2abe2de9f04fa44a20f0004890450c46814687b004d89c
:020000040800f2
:2099e000002308604b6000251de09f4a90454fd820f0004500289d499d4f25f00f0524ddb1
:020000040800f2
:209a0000fdf752fdbd42064611d09a49fdf74cfd014605463046fdf747fd9649fdf744fd63
:020000040800f2
:209a2000256001256060284607b0bde8f08f9249fdf73afd91490646fdf736fd014605468d
:020000040800f2
:209a40003046fdf731fd8d49e8e7fdf72ffdbd4206460fd08749fdf729fd0146054630468d
:020000040800f2
:209a6000fdf722fd8349fdf721fd256060604ff0ff35d8e78049fdf719fd80490646fdf7a2
:020000040800f2
:209a800015fd014605463046fdf70efd7b49eae77b4a904500f2948020f0004630467949ea
:020000040800f2
:209aa000fdf70cfe4ff07c51fdf700fdfdf7ccff0546fdf7affd6d498246fdf7fffd01464c
:020000040800f2
:209ac0003046fdf7f1fc6b4907465046fdf7f6fd014606463846fdf7e7fc1f2d09dc6a4ae4
:020000040800f2
:209ae000691e52f8212029f0004323f0ff03934207d1c0f3c753c3ebd853082b4feae85be1
:020000040800f2
:209b000001dc206026e05c495046fdf7d7fd064601463846fdf7c8fc014680463846fdf797
:020000040800f2
:209b2000c3fc3146fdf7c0fc064654495046fdf7c5fd3146fdf7b8fc014606464046fdf7de
:020000040800f2
:209b4000b3fcc0f3c753abeb030bbbf1190f18dc47462060d4f8008038464146fdf7a4fc2b
:020000040800f2
:209b60003146fdf7a1fcb9f1000f6060bff65baf08f1004800f10040c4f8008060606d4288
:020000040800f2
:209b800051e750464149fdf799fd064601464046fdf78afc074601464046fdf785fc31464a
:020000040800f2
:209ba000fdf782fc06463a495046fdf787fd3146fdf77afc064601463846fdf775fca0e778
:020000040800f2
:209bc000b8f1ff4f05d30146fdf76efc6060206009e74feae856863ea8ebc6584046fdf77b
:020000040800f2
:209be00033fffdf717fd014603904046fdf75cfc4ff08741fdf762fd0746fdf725fffdf7cc
:020000040800f2
:209c000009fd0146049005463846fdf74dfc4ff08741fdf753fd00210590fdf7e3fef0b1e6
:020000040800f2
:209c200000212846fdf7defe002814bf01230223184a21460192022203a80092324600f05c
:020000040800f2
:209c40002bf8b9f1000f0546bff6edae236803f100432360636803f1004363608fe70323e7
:020000040800f2
:209c6000e6e700bfd80f493fe3cb1640800fc93fd00fc93f434435370044353708a3852e66
:020000040800f2
:209c8000800f494384f9223f3cbc000800a3852e32318d24bcbc00082de9f04fdbb002926d
:020000040800f2
:209ca0000493649aac4b059053f8223000910193049b013b0393029b1a1dc0f29980dc1eb7
:020000040800f2
:209cc00048bf1c1de41000254ff0000b671cfb000693029b039aa3ebc707019ba4eb0208ff
:020000040800f2
:209ce00003eb0209659b1eae03eb880a4d4540f38180049a1eab03eb82054ff00009002312
:020000040800f2
:209d00000df58c7a019a914540f39a8013460aaa02eb83030893659b03eb8403019c0793b6
:020000040800f2
:209d20000df12808464625464ff087495aab03eb840353f850bc0df58c7a002d00f38580f1
:020000040800f2
:209d40003946584600f046fa4ff078510546fdf7b5fc00f091fa4ff08241fdf7affc01465b
:020000040800f2
:209d60002846fdf7a1fb0546fdf76efe0646fdf751fc01462846fdf797fb002f814640f349
:020000040800f2
:209d80008180621e0aab53f82250c7f1080145fa01f31e448b40ed1a0aab43f82250c7f18e
:020000040800f2
:209da00007031d41002d7add002292460136944200f3aa80002f05dd012f00f0b680022ffb
:020000040800f2
:209dc00000f0bd80022d6ad149464ff07e50fdf76bfb8146baf1000f61d039464ff07e50b8
:020000040800f2
:209de00000f0f8f901464846fdf75efb814656e0002468e718eb050f07d45af82500fdf793
:020000040800f2
:209e000009fc46f8040b013570e75846f9e70793059b5bf8041d53f82800fdf74ffc01463e
:020000040800f2
:209e20003046fdf743fb0646079b08f10108039a9045ecdd4af8046b09f10109043561e719
:020000040800f2
:209e4000ab461e464ff00008f1e74ff06e515846fdf734fcfdf7f8fdfdf7dcfb49460990f2
:020000040800f2
:209e6000fdf72cfc01465846fdf71efbfdf7ecfd013d46f8040b5af825100998fdf716fb3f
:020000040800f2
:209e800083465ae705d1631e0aaa52f82350ed1188e74ff07c51fdf7c3fd054690bb00210c
:020000040800f2
:209ea0004846fdf79ffd002800f090800022631e01998b424ada002a76d0013c0aab53f881
:020000040800f2
:209ec0002430083f002bf8d039464ff07e5000f081f9a24607464ff06e590df58c78baf112
:020000040800f2
:209ee000000f80f2a18027460022002fc0f2cb8046a990464ff0000a184b01eb870ba4eb87
:020000040800f2
:209f00000709b4e002254fe758f8043bbaf1000f08d123b1c3f5807348f8043c01239a461b
:020000040800f2
:209f2000013244e7c3f1ff03f6e7621e0aab53f8223003f07f030aa941f8223042e7621e02
:020000040800f2
:209f40000aab53f8223003f03f03f4e70aa951f82310013b0a43abe7d4bf0008e0bf000813
:020000040800f2
:209f6000013352f8041d0029fad0049a1ea9a218661c01eb82051c440df58c79b442fff6e9
:020000040800f2
:209f8000cfae079bab4653f82600fdf743fb4ff0000a4ff000082860039b9a4507dd49f854
:020000040800f2
:209fa000268004350136e9e70123089ad9e7059b5bf8040953f82a10fdf780fb0146404674
:020000040800f2
:209fc000fdf774fa0af1010a8046e5e7069b029a4846991a00f0fef84ff087418046fdf762
:020000040800f2
:209fe0001ffdf8b14ff06e514046fdf767fbfdf72bfdfdf70ffb4ff087418146fdf75efb8d
:020000040800f2
:20a0000001464046fdf750fafdf71efd0aab43f82400484601340837fdf716fd0aab43f819
:020000040800f2
:20a02000240051e74046f7e70aab53f82a00fdf7f1fa3946fdf742fb494648f82a00384630
:020000040800f2
:20a04000fdf73cfb0af1ff3a074648e753f8040b5bf8041b03920293fdf730fb0146404643
:020000040800f2
:20a06000fdf724fadde9023280460af1010a01998a4501dcca45e9dd5aab03eb890949f827
:020000040800f2
:20a08000a08c013f31e7649b022b07dc002b4edc2ed006f007005bb0bde8f08f649b032b81
:020000040800f2
:20a0a000f7d10df1c80b0beb8407b846a246baf1000f49dca146b9f1010f60dc0020012c97
:020000040800f2
:20a0c00076dc329a339b002d78d100990a600a464b609060dde757f82410fdf7e7f9013cd8
:020000040800f2
:20a0e000002cf8da0db100f10040009b1860d0e7002032aff4e757f82810fdf7d7f908f189
:020000040800f2
:20a10000ff38b8f1000ff6daadb100f10043009a014613603298fdf7c7f94ff0010844454b
:020000040800f2
:20a120000bda0db100f10040009b5860b1e7a046002032afe5e70346e9e757f8041ffdf72e
:020000040800f2
:20a14000b5f908f10108eae7d8f8003058f8042c1946104602930192fdf7a8f9019a0146aa
:020000040800f2
:20a1600081461046fdf7a0f9029b0af1ff3a1946fdf79cf948f80409c8f8009097e757f812
:020000040800f2
:20a18000043cd7f800a0184651460193fdf78ef9019b014680461846fdf786f95146fdf707
:020000040800f2
:20a1a00085f947f8040909f1ff39c7f8008082e75bf82410fdf77af9013c80e7009902f1dd
:020000040800f2
:20a1c000004203f100430a604b600a4600f100407fe700bf38b5c0f3c7540d46034620f0e4
:020000040800f2
:20a1e000004184b941b34ff09841fdf767fa1a4bc0f3c7549d42a4f1190406dabde83840bf
:020000040800f2
:20a20000c00f00f02bb8ff2c08d04cf250339d4209ddbde83840c00f00f026b80146fdf71e
:020000040800f2
:20a2200045f9034608e02b19fe2bf2dc002b05dd20f0ff4040eac353184638bd13f1180f5a
:020000040800f2
:20a24000dcdb193320f0ff404ff04c5140eac350fdf734fae5e700bfb03cffff10b14ff0fc
:020000040800f2
:20a26000004070470020704708b1024870474ff0ff407047000080ff38b5c0f3c7537f3b2e
:020000040800f2
:20a28000162b014620f0004519dc002b024608da00281bda002d0e4908bf4ff00041084661
:020000040800f2
:20a2a00038bd0c4818410842f9d00029bebf4ff4000141fa03f3d21822ea0001efe7b5f15b
:020000040800f2
:20a2c000ff4fecd3fdf7f2f80146e8e70021e6e7000080bfffff7f00dd11000800000000dd
:020000040800f2
:20a2e000456173794d6567612d76332e3000616c7475736d657472756d2e6f726700312e86
:020000040800f2
:20a30000392e313800006d616e756661637475726572202020202025730a70726f64756391
:020000040800f2
:20a32000742020202020202020202025730a73657269616c2d6e756d6265722020202025ec
:020000040800f2
:20a34000750a63757272656e742d666c6967687420202025750a6c6f672d666f726d6174d4
:020000040800f2
:20a360002020202020202025750a6c6f672d73706163650920256c750a70726f6772616dad
:020000040800f2
:20a380002d73706163652020202025750a616c7469747564652d3332202020202020310a77
:020000040800f2
:20a3a00000736f6674776172652d76657273696f6e20252e38730a0053796e7461782065cb
:020000040800f2
:20a3c00072726f720a0065626f6f7400636d6400252d3230732025730a005265706f7274fc
:020000040800f2
:20a3e00020696e20666565743a2025640a004265657065722073657474696e673a20256461
:020000040800f2
:20a400000a005079726f2074696d653a2025640a0049676e697465206d6f64653a202564c4
:020000040800f2
:20a420000a004d617820666c69676874206c6f673a202564206b420a00506164206f7269b3
:020000040800f2
:20a44000656e746174696f6e3a2025640a00416363656c2063616c202b31673a202564209f
:020000040800f2
:20a460002d31673a2025640a00494d552063616c20616c6f6e67202564206163726f73736a
:020000040800f2
:20a48000202564207468726f7567682025640a0041706f676565206c6f636b6f75743a2073
:020000040800f2
:20a4a0002564207365636f6e64730a0041706f6765652064656c61793a202564207365633c
:020000040800f2
:20a4c0006f6e64730a004d61696e206465706c6f793a202564206d65746572730a004f722e
:020000040800f2
:20a4e00069656e7420616e74656e6e6120257320616e642070726573732061206b65792e37
:020000040800f2
:20a500002e2e000d0a0043616c6962726174696e672e2e2e005361766564004e6f746869e9
:020000040800f2
:20a520006e6720746f2073617665004e3043414c4c0053746f72616765206d75737420629a
:020000040800f2
:20a540006520656d707479206265666f7265206368616e67696e67206c6f672073697a6518
:020000040800f2
:20a5600000466c69676874206c6f67206d6178202575206b420a00757000646f776e00493e
:020000040800f2
:20a580006e76616c696420616363656c3a207570202825642920646f776e20282564290a10
:020000040800f2
:20a5a00000436f6e6669672076657273696f6e3a2025642e25640a002532643a2077636824
:020000040800f2
:20a5c000616e202530387820616c61726d202535642025730a00446f4974006d61696e00a5
:020000040800f2
:20a5e00064726f6775650049676e697465723a20253673205374617475733a2025730a003b
:020000040800f2
:20a6000069676e6974657200756e6b6e6f776e00726561647900616374697665006f706563
:020000040800f2
:20a620006e00776169745f616464722025640a0050726573737572653a2020202025386c6e
:020000040800f2
:20a64000752025386c640a0054656d70657261747572653a2025386c752025386c640a00b1
:020000040800f2
:20a66000416c7469747564653a20256c640a006d73353630372072657365727665643a20b9
:020000040800f2
:20a6800025750a006d73353630372073656e733a2025750a006d7335363037206f66663a46
:020000040800f2
:20a6a0002025750a006d7335363037207463733a2025750a006d73353630372074636f3a6a
:020000040800f2
:20a6c0002025750a006d733536303720747265663a2025750a006d73353630372074656d1d
:020000040800f2
:20a6e0007073656e733a2025750a006d7335363037206372633a2025750a006d73353630b0
:020000040800f2
:20a700003700424d493038383a202537642025376420253764202537642025376420253774
:020000040800f2
:20a72000640a00626d69303838004d4d43353938333a2025642025642025640a006d6d63a1
:020000040800f2
:20a7400035393833004144584c3337352076616c75652025642025642025642073656c6656
:020000040800f2
:20a76000207465737420256c64206d696e20256c64206d617820256c640a006164786c330a
:020000040800f2
:20a780003735007469636b3a2025356c7520413a2025356420423a2025356420433a202538
:020000040800f2
:20a7a000356420443a202535642064726f6775653a20253564206d61696e3a2025356420c9
:020000040800f2
:20a7c000626174743a202535642070626174743a202535642074656d703a202535640a006b
:020000040800f2
:20a7e00053746f726167652073697a653a20256c640a0053746f726167652065726173654b
:020000040800f2
:20a8000020756e69743a20256c640a00446574656374656420636869707320312073697adf
:020000040800f2
:20a820006520256c640a007265706f7274004e6f207375636820666c696768743a20256cdf
:020000040800f2
:20a84000640a00457261736564004661696c656420746f20657261736500666c6967687440
:020000040800f2
:20a8600020256c6420737461727420257820656e642025780a00736c6f742025642020737c
:020000040800f2
:20a880007461727420257820656e642025780a00646f6e65006c6f6700666c6967687400bc
:020000040800f2
:20a8a000436f6d70616e696f6e2072756e6e696e673a2025640a006465766963653a2025f7
:020000040800f2
:20a8c000640a75706461746520706572696f643a2025640a6368616e6e656c733a202564c8
:020000040800f2
:20a8e0000a646174613a002025357500636f6d70616e696f6e00257325730049676e69749c
:020000040800f2
:20a9000065723a202564205374617475733a2025730a005079726f2d636f756e743a20255e
:020000040800f2
:20a92000640a005079726f202532643a20003c64697361626c65643e0025366c64200020ad
:020000040800f2
:20a94000202020202020003c6e3e2000696e76616c6964207079726f206368616e6e656c65
:020000040800f2
:20a9600020256c750a00696e76616c6964207079726f206669656c642025730a00616f5fc1
:020000040800f2
:20a980007079726f5f6d616e75616c2025640a007079726f00616363656c206c65737320a4
:020000040800f2
:20a9a000286d2f7373202a2031362900616363656c206772656174657220286d2f73732007
:020000040800f2
:20a9c0002a20313629007370656564206c65737320286d2f73202a203136290073706565b7
:020000040800f2
:20a9e00064206772656174657220286d2f73202a2031362900686569676874206c65737348
:020000040800f2
:20aa000020286d2900686569676874206772656174657220286d29006f7269656e74206cda
:020000040800f2
:20aa2000657373202864656729006f7269656e74206772656174657220286465672900747a
:020000040800f2
:20aa4000696d65206c657373202873202a20313030290074696d652067726561746572202c
:020000040800f2
:20aa60002873202a2031303029007374617465206c657373007374617465206772656174cb
:020000040800f2
:20aa80006572206f7220657175616c00617363656e64696e670064657363656e64696e67e6
:020000040800f2
:20aaa000006166746572206d6f746f720064656c6179206265666f726520666972696e67f2
:020000040800f2
:20aac000202873202a203130302900696e66006e616e00286e756c6c2900000008200800e1
:020000040800f2
:20aae000d514000818ab00080d2400081fab0008d517000827ab00087d1800083cab000835
:020000040800f2
:20ab0000551400084bab00084514000855ab000800000000000000003f0048656c70005441
:020000040800f2
:20ab2000005461736b730045203c30206f66662c2031206f6e3e004563686f007220656253
:020000040800f2
:20ab40006f6f74005265626f6f7400760056657273696f6e00580053776974636820746f0f
:020000040800f2
:20ab600020626f6f74206c6f616465720000000067ac0008e91f0008491a000882ac00089e
:020000040800f2
:20ab8000b91f0008351a00089dac0008851f0008211a0008c3ac0008691e0008ed1900082a
:020000040800f2
:20aba000e8ac0008291e0008d919000819ad0008bd1d0008c119000837ad0008951d000878
:020000040800f2
:20abc000ad1900086cad0008457100089170000882ad0008691d0008991900089dad0008ee
:020000040800f2
:20abe0003d1d000885190008cead00080d1d00087119000808ae00082520000800000000fb
:020000040800f2
:20ac00000fae0008711b00080000000021ae000835190008000000000000000000000000ae
:020000040800f2
:20ac2000000000002d1b000834ac0008000000000000000063203c7661723e203c76616cf7
:020000040800f2
:20ac400075653e0053657420636f6e66696720283f20666f722068656c702c207320746fa1
:020000040800f2
:20ac60002073686f7729006d203c6d65746572733e004d61696e206465706c6f7920286d4c
:020000040800f2
:20ac8000290064203c64656c61793e0041706f6765652064656c617920287329004c203c72
:020000040800f2
:20aca0007365636f6e64733e0041706f67656520646574656374206c6f636b6f7574202814
:020000040800f2
:20acc00073290061203c2b673e203c2d673e00416363656c2063616c696220283020666fbd
:020000040800f2
:20ace00072206175746f29006f203c3020616e74656e6e612075702c203120616e74656e28
:020000040800f2
:20ad00006e6120646f776e3e00506164206f7269656e746174696f6e006c203c73697a65ea
:020000040800f2
:20ad20003e00466c69676874206c6f672073697a6520286b42290069203c30206475616c61
:020000040800f2
:20ad40002c20312061706f6765652c2032206d61696e2c203320626f6f737465723e00497e
:020000040800f2
:20ad6000676e69746572206d6f64650050203c6e2c3f3e005079726f206368616e6e656c1f
:020000040800f2
:20ad8000730049203c7469636b733e005079726f20666972696e672074696d650062203c69
:020000040800f2
:20ada00076616c3e0042656570657220746f6e65202866726571203d20312f322028323436
:020000040800f2
:20adc00065362f333229202f20626565700075203c30206d65746572732c20312066656592
:020000040800f2
:20ade000743e00556e69747320746f207265706f72742068656967687420616674657220e4
:020000040800f2
:20ae00006c616e64696e6700730053686f77007700577269746520746f20656570726f6d14
:020000040800f2
:20ae2000003f0048656c70000008014009000000000801400a0000000c00002008a60008c3
:020000040800f2
:20ae400010a6000816a600081da600088529000864ae0008752a00089fae000800000000d9
:020000040800f2
:20ae60000000000069203c6b65793e207b6d61696e7c64726f6775657d00466972652069b8
:020000040800f2
:20ae8000676e697465722e203c6b65793e20697320646f6974207769746820442649007429
:020000040800f2
:20aea00000546573742069676e6974657200000001020000003001400304000000380040ed
:020000040800f2
:20aec0000506000000540040030400000058004081390008e0ae00080000000000000000dc
:020000040800f2
:20aee0004200446973706c6179204d53353630372064617461000000a53a000808af000848
:020000040800f2
:20af00000000000000000000490053686f7720424d493038382073746174757300000000eb
:020000040800f2
:20af2000193e000830af000800000000000000004d0053686f77204d4d4335393833207374
:020000040800f2
:20af40007461747573000000b540000858af000800000000000000004100446973706c6116
:020000040800f2
:20af600079204144584c33373520646174610000b943000880af000800000000000000007b
:020000040800f2
:20af80006100446973706c61792063757272656e74204144432076616c75657300000000bf
:020000040800f2
:20afa00055460008c8af0008e9460008d7af0008a5480008ecaf00087d48000804b0000889
:020000040800f2
:20afc0000000000000000000660053686f772073746f726167650065203c626c6f636b3e4b
:020000040800f2
:20afe0000044756d7020666c617368007a203c626c6f636b3e004572617365203c626c6fe5
:020000040800f2
:20b00000636b3e005a203c6b65793e00457261736520616c6c2e203c6b65793e2069732071
:020000040800f2
:20b02000646f6974207769746820442649000302340c242c0b1a144c2eec00007d9500006b
:020000040800f2
:20b040005a8a0000ed7f00008a780000cf720000236e0000336a0000cd660000d0630000c9
:020000040800f2
:20b0600025610000bc5e00008b5c0000885a0000ac580000f256000055550000d25300004c
:020000040800f2
:20b08000665200000e510000c84f0000924e00006b4d0000514c0000434b0000414a000034
:020000040800f2
:20b0a00048490000594800007247000094460000bd450000ed44000023440000604300008e
:020000040800f2
:20b0c000a3420000eb410000394100008b400000e23f00003d3f00009d3e0000003e000064
:020000040800f2
:20b0e000673d0000d23c0000403c0000b23b0000263b00009e3a0000183a000096390000db
:020000040800f2
:20b1000016390000983800001d380000a43700002e370000b936000047360000d735000003
:020000040800f2
:20b1200068350000fc3400009134000029340000c13300005c330000f832000096320000ab
:020000040800f2
:20b1400035320000d6310000783100001b310000c0300000663000000d300000b62f0000e4
:020000040800f2
:20b16000602f00000a2f0000b62e0000632e0000122e0000c12d0000712d0000222d000077
:020000040800f2
:20b18000d52c0000882c00003c2c0000f12b0000a62b00005d2b0000152b0000cd2a0000e6
:020000040800f2
:20b1a000862a0000402a0000fa290000b5290000702900002c290000e9280000a6280000a7
:020000040800f2
:20b1c0006428000022280000e1270000a02700006027000020270000e1260000a32600002c
:020000040800f2
:20b1e0006426000027260000ea250000ad2500007025000035250000f9240000be240000a9
:020000040800f2
:20b20000842400004924000010240000d62300009d230000652300002c230000f52200003e
:020000040800f2
:20b22000bd220000862200004f22000019220000e3210000ad21000078210000432100000c
:020000040800f2
:20b240000e210000da200000a6200000722000003f2000000c200000d91f0000a71f000024
:020000040800f2
:20b26000741f0000431f0000111f0000e01e0000af1e00007e1e00004e1e00001d1e00009b
:020000040800f2
:20b28000ed1d0000be1d00008e1d00005f1d0000301d0000021d0000d31c0000a51c000086
:020000040800f2
:20b2a000771c00004a1c00001c1c0000ef1b0000c21b0000951b0000691b00003d1b0000ea
:020000040800f2
:20b2c000111b0000e51a0000b91a00008e1a0000631a0000381a00000d1a0000e2190000d7
:020000040800f2
:20b2e000b81900008e190000641900003a19000011190000e7180000be180000951800005a
:020000040800f2
:20b300006c180000441800001b180000f3170000cb170000a31700007b1700005417000077
:020000040800f2
:20b320002d17000005170000de160000b7160000911600006a160000441600001e16000037
:020000040800f2
:20b34000f8150000d2150000ac15000086150000611500003c15000017150000f2140000a4
:020000040800f2
:20b36000cd140000a8140000841400005f1400003b14000017140000f3130000cf130000c3
:020000040800f2
:20b38000ac1300008813000065130000411300001e130000fb120000d8120000b612000097
:020000040800f2
:20b3a00093120000711200004e1200002c1200000a120000e8110000c6110000a411000026
:020000040800f2
:20b3c0008311000061110000401100001f110000fe100000dd100000bc1000009b10000074
:020000040800f2
:20b3e0007a1000005a1000003910000019100000f90f0000d90f0000b80f0000990f000088
:020000040800f2
:20b40000790f0000590f00003a0f00001a0f0000fb0e0000db0e0000bc0e00009d0e000063
:020000040800f2
:20b420007e0e00005f0e0000410e0000220e0000030e0000e50d0000c70d0000a80d000008
:020000040800f2
:20b440008a0d00006c0d00004e0d0000300d0000120d0000f50c0000d70c0000b90c00007c
:020000040800f2
:20b460009c0c00007f0c0000610c0000440c0000270c00000a0c0000ed0b0000d00b0000c0
:020000040800f2
:20b48000b40b0000970b00007a0b00005e0b0000410b0000250b0000090b0000ed0a0000d6
:020000040800f2
:20b4a000d10a0000b50a0000990a00007d0a0000610a0000450a00002a0a00000e0a0000c2
:020000040800f2
:20b4c000f3090000d7090000bc090000a1090000860900006b090000500900003509000087
:020000040800f2
:20b4e0001a090000ff080000e4080000ca080000af080000950800007a0800006008000026
:020000040800f2
:20b50000460800002b08000011080000f7070000dd070000c3070000a9070000900700009e
:020000040800f2
:20b52000760700005c070000430700002907000010070000f6060000dd060000c4060000f1
:020000040800f2
:20b54000aa06000091060000780600005f060000460600002d06000014060000fc05000027
:020000040800f2
:20b56000e3050000ca050000b205000099050000810500006805000050050000380500003a
:020000040800f2
:20b580001f05000007050000ef040000d7040000bf040000a70400008f0400007704000031
:020000040800f2
:20b5a0005f04000048040000300400001804000001040000e9030000d2030000ba03000009
:020000040800f2
:20b5c000a30300008c030000740300005d030000460300002f0300001803000001030000c5
:020000040800f2
:20b5e000ea020000d3020000bc020000a60200008f02000078020000620200004b02000068
:020000040800f2
:20b60000340200001e02000008020000f1010000db010000c5010000ae01000098010000ee
:020000040800f2
:20b62000820100006c01000056010000400100002a01000014010000fe000000e80000005c
:020000040800f2
:20b64000d3000000bd000000a7000000910000007c00000066000000510000003b000000b4
:020000040800f2
:20b660002600000011000000fcffffffe7ffffffd2ffffffbcffffffa7ffffff92fffffffb
:020000040800f2
:20b680007dffffff68ffffff53ffffff3effffff29ffffff14ffffff00ffffffebfeffff25
:020000040800f2
:20b6a000d6feffffc1feffffadfeffff98feffff84feffff6ffeffff5bfeffff46feffff3a
:020000040800f2
:20b6c00032feffff1dfeffff09fefffff5fdffffe1fdffffccfdffffb8fdffffa4fdffff39
:020000040800f2
:20b6e00090fdffff7cfdffff68fdffff54fdffff40fdffff2cfdffff18fdffff04fdffff22
:020000040800f2
:20b70000f0fcffffddfcffffc9fcffffb5fcffffa2fcffff8efcffff7afcffff67fcfffffd
:020000040800f2
:20b7200053fcffff40fcffff2dfcffff19fcffff06fcfffff2fbffffdffbffffccfbffffc0
:020000040800f2
:20b74000b9fbffffa5fbffff92fbffff7ffbffff6cfbffff59fbffff46fbffff33fbffff74
:020000040800f2
:20b7600020fbffff0dfbfffffafaffffe7faffffd5faffffc2faffffaffaffff9cfaffff17
:020000040800f2
:20b780008afaffff77faffff64faffff52faffffb95b0008a8b70008e15a0008b4b70008d9
:020000040800f2
:20b7a00000000000000000006c004c697374206c6f67730064203c666c696768742d6e755e
:020000040800f2
:20b7c0006d6265723e0044656c65746520666c69676874005d6c0008e4b700080000000020
:020000040800f2
:20b7e000000000004c00436f6d70616e696f6e206c696e6b2073746174757300613c00002a
:020000040800f2
:20b800000100020095a90008613e000002000400aca90008733c000004000600c6a90008ad
:020000040800f2
:20b82000733e000008000800dca90008683c000010000a00f5a90008683e000020000c0084
:020000040800f2
:20b8400005aa00086f3c000040000e0018aa00086f3e0000800010002aaa0008743c0000a5
:020000040800f2
:20b86000000114003faa0008743e00000002180053aa0008663c0000004020006aaa0008d3
:020000040800f2
:20b88000663e3d000080210075aa0008410000000004ff008caa0008440000000008ff0032
:020000040800f2
:20b8a00096aa00086d00000000102200a1aa00086400000000201c00adaa0008000000004f
:020000040800f2
:20b8c0000000ff00000000000100021002000410040006100800081010000a1020000c10a0
:020000040800f2
:20b8e00040000e1080001010000112100002141000201610004018080080190800101a1080
:020000040800f2
:20b90000000000000000000000000000000000100000000000000000b9340332b7f4ad1489
:020000040800f2
:20b9200010db1ab30892540e0d307d951447ba1a66088f4d26adc66df598bf85e2b74511c5
:020000040800f2
:20b94000ca96853d92bd1debfca11860dcef52163c92ae220bb8c1b4839d2d5b0562da1c4b
:020000040800f2
:20b96000304c7e8f4e8bb25b16f4529f8b56a512fbd4827643ed8af08fe7f9311565191809
:020000040800f2
:20b9800050f19bd94a13eeb4284cf0a686c1251f035fc270cb9e4916e642889c44eb201453
:020000040800f2
:20b9a000b0650836ad6ea58585f0ca14e2fd031a0b899979d5b13d09d8da973a35ebcf10ac
:020000040800f2
:20b9c000ac363f5e73bb38cf3e6752fa44afba1501000000000000000500000000000000fa
:020000040800f2
:20b9e00019000000000000007d000000000000007102000000000000350c000000000000fd
:020000040800f2
:20ba0000093d0000000000002d31010000000000e1f505000000000065cd1d000000000057
:020000040800f2
:20ba2000f902950000000000dd0ee90200000000514a8d0e000000009573c2480000000058
:020000040800f2
:20ba4000e941cc6b010000008d49fd1a07000000c16ff28623000000c52ebca2b1000000c3
:020000040800f2
:20ba6000d9e9ac2d780300003d9160e45811000031d6e275bc560000f52e6e4daeb1010087
:020000040800f2
:20ba8000c9ea268367780800ed95c28f055a2a00a1edccce1bc2d30025a4000a8bca2204e1
:020000040800f2
:20baa00000000000000000000000000000000000000000409559695955555455155555562e
:020000040800f2
:20bac000040515411054554045515544404550445055554500400040400444966555565584
:020000040800f2
:20bae00045404554514115405591555555554051050100000000000001000000000000006f
:020000040800f2
:20bb00000000000000000020345065c05fc9a652bb13cbaec440c21806c8df7100d5a87c00
:020000040800f2
:20bb2000f56f0fda58fc27136e4756357d24206502c7e768e48ca41de9e60268d7cd396104
:020000040800f2
:20bb40007977fcc2405bef16798cde43ffa751f991f3b278f5bdbe11e857e9d6e8bee87b4b
:020000040800f2
:20bb6000b054ac8f848d751bea23a499e9f9d38bb7a3714061da3e15cee33ecb73f948084c
:020000040800f2
:20bb80008c97b427d51b7010a2bfefb9eb8532154db44db49bbb6f1996b6076cf8e7eead5e
:020000040800f2
:20bba00036d9b4f59135ae13222218af4e6a684d91daaa3d4f40741e9fbd9ee006a1c09882
:020000040800f2
:20bbc00057c2a7fda40e90170e7d497173e3208fb220d87605143b12853d7434811343b08e
:020000040800f2
:20bbe000ad297a5f27f4351c54455454455505040010041014044000000001405555154189
:020000040800f2
:20bc00005404000044000100000000404100004450444550540055555455655100400040bc
:020000040800f2
:20bc200001000001000501001154515154555505000000000000000000000000000fc93fdb
:020000040800f2
:20bc4000000f494000cb9640000fc9400053fb4000cb164100ed2f41000f49410031624119
:020000040800f2
:20bc600000537b41003a8a4100cb9641005ca34100edaf41007ebc41000fc94100a0d541a7
:020000040800f2
:20bc80000031e24100c2ee410053fb4100f20342003a0a420083104200cb164200141d42a8
:020000040800f2
:20bca000005c234200a5294200ed2f4200363642007e3c4200c74242000f4942a200000024
:020000040800f2
:20bcc000f9000000830000006e0000004e000000440000001500000029000000fc000000ae
:020000040800f2
:20bce0002700000057000000d1000000f500000034000000dd000000c0000000db00000054
:020000040800f2
:20bd00006200000095000000990000003c000000430000009000000041000000fe00000045
:020000040800f2
:20bd20005100000063000000ab000000de000000bb000000c500000061000000b70000002e
:020000040800f2
:20bd4000240000006e0000003a000000420000004d000000d2000000e000000006000000d0
:020000040800f2
:20bd6000490000002e000000ea00000009000000d1000000920000001c000000fe000000dc
:020000040800f2
:20bd80001d000000eb0000001c000000b100000029000000a70000003e000000e8000000d8
:020000040800f2
:20bda0008200000035000000f50000002e000000bb0000004400000084000000e90000003d
:020000040800f2
:20bdc0009c0000007000000026000000b40000005f0000007e000000410000003900000026
:020000040800f2
:20bde00091000000d600000039000000830000005300000039000000f40000009c00000004
:020000040800f2
:20be0000840000005f0000008b000000bd000000f9000000280000003b0000001f0000007c
:020000040800f2
:20be2000f800000097000000ff000000de00000005000000980000000f000000ef000000fb
:020000040800f2
:20be40002f000000110000008b0000005a0000000a0000006d0000001f0000006d000000ba
:020000040800f2
:20be6000360000007e000000cf00000027000000cb00000009000000b70000004f0000003e
:020000040800f2
:20be8000460000003f000000660000009e0000005f000000ea0000002d000000750000002e
:020000040800f2
:20bea00027000000ba000000c7000000eb000000e5000000f10000007b0000003d00000061
:020000040800f2
:20bec0000700000039000000f70000008a0000005200000092000000ea0000006b00000068
:020000040800f2
:20bee000fb0000005f000000b10000001f0000008d0000005d0000000800000056000000d0
:020000040800f2
:20bf0000030000003000000046000000fc0000007b0000006b000000ab000000f00000002b
:020000040800f2
:20bf2000cf000000bc000000200000009a000000f4000000360000001d000000a9000000cc
:020000040800f2
:20bf4000e300000091000000610000005e000000e60000001b000000080000006500000040
:020000040800f2
:20bf600099000000850000005f00000014000000a000000068000000400000008d0000005b
:020000040800f2
:20bf8000ff000000d8000000800000004d000000730000002700000031000000060000002c
:020000040800f2
:20bfa000060000001500000056000000ca00000073000000a8000000c90000006000000002
:020000040800f2
:20bfc000e20000007b000000c00000008c0000006b00000004000000070000000900000039
:020000040800f2
:20bfe0000000c93f0000f0390000da370000a2330000842e0000502b0000c2270000d02222
:020000040800f2
:20c000000000c41f0000c61b0000441700000300e525000829260008f9250008010000006e
:020000040800f2
:08c0200000c20100000008004d
:00000001ff
